:020000040000fa
:080000000414040000000000dc
:020000040000fa
:1004000000000000000000000000000000000000ec
:1004100000000000000000000000000000000000dc
:1004200000000000000000000000000000000000cc
:1004300000000000000000000000000000000000bc
:10280000ffffff00ffffff000f212100807f24005a
:1028100000018800000000000a0007001100070006
:10282000000020000000e000020032000000020072
:1028300000000000fc4b0200000000000040da0035
:102840000000fe004440a900c08020000000e0001d
:102850000300320000002000a00188004440a800ce
:10286000000006004040250001002000160037004f
:1028700062004000e0804800910188009001ba00a9
:1028800062004000e0804800910188009002ba0098
:1028900062004000e08048000002eb006028e10098
:1028a00005003a008301e9000700330003800900b6
:1028b0000059eb00040037006128e10001003200fc
:1028c0000082eb0005000700910188001001ba00aa
:1028d0000200e000e6ff3a000000050091018800d8
:1028e0008002780062004000e08048003559ba005c
:1028f0008301e900080032002559ba008301e9008c
:10290000050032000400e000f4ff320015d9ba00df
:102910008301e900f1ff3a0000000600e6500400e0
:10292000000000004c51040000000000889fbe0021
:10293000e30440000900a100808f54004a003600e3
:10294000e38f540001003e0049002000e246800071
:102950000200e00002003200820078000c00370024
:10296000e18d200003003700908f540023003600d3
:102970008080e800110078000000e000faff3a00d3
:102980000f003700908f54001c0036008080e80054
:10299000110078000000e000faff3a001201780010
:1029a000e18d200003003700908f540013003600a3
:1029b0008080e80011007800820f5000faff3a0092
:1029c000d8468000890f54000100310009047800c6
:1029d00008007800620007000000e00004003a00f0
:1029e000890f5400200032000804d100f5ff3700a1
:1029f000081878001f000700d4ff37001101780085
:102a00009201780064805100890f5000030031006a
:102a1000120090008008780007003700090041008c
:102a2000800878009201900013009800110078004f
:102a30001288140009097800910078000100e00074
:102a400005003200110090000000e000020032009a
:102a50000180e800010037000000eb00e04688003c
:102a60000280e800010037000000eb004f04be00c8
:102a7000000006000000e000310032008080e90024
:102a800091027800e38f52002d0036000508a30064
:102a90002b003a00f24680000200e0000200320003
:102aa000828f50000400310002087800f14688004f
:102ab0001600370003017800920190000300e00047
:102ac00002003200818f5100faff390012027800b3
:102ad00004004100808f500019003900810f500020
:102ae00003003a0005094200820078000700370021
:102af0000300e0000300320005804000808f510099
:102b00000f00390093009800110198001101900006
:102b10000200e0000a00320011804000820f5000e5
:102b200007003a00c08d20000008eb001100900063
:102b3000110178009008410010009000900098006a
:102b4000000006008001eb00020037008171780070
:102b50008301e800828f5100fcff3a00000006006c
:102b60000000e0000300340004000700e10f400013
:102b700001003a000000eb0000000600889fbe0044
:102b800080047800d808e20004003a000000eb005e
:102b9000100007000000e0000a003500c046800079
:102ba0000900e00002003a00000478000600370047
:102bb0000004780009004000060007000000e00063
:102bc00001003d000084eb00080078004f04be00c7
:102bd00000000600800078000000e00004003a00d9
:102be00000a12000c04688000101780006003700df
:102bf0000081eb0000212100808f500002003e0088
:102c0000c14688000001eb000200780000000600c9
:102c10006022b800060220000000d0008180d200af
:102c20000482d2008582d2000000a000020252007d
:102c300083825a00030031000202420083824a006c
:102c40000000a1000603e900f3ff3a0000000600bf
:0c2c5000efff07000400be0000000600bb
:020000040000fa
:020000040005f5
:0457f800fe9300001c
:020000040000fa
:020000040005f5
:0457fc007f3e0000ec
:020000040000fa
:100008005e5400005e5400005e5400005e54000020
:100018005e5400005e5400005e5400005e54000010
:100028005e5400005e5400005e5400005e54000000
:100038005e5400005e5400005e5400005e540000f0
:100048005e5400005e5400005e5400005e540000e0
:100058005e5400005e5400005e5400005e540000d0
:100068005e5400005e5400005e5400005e540000c0
:100078005e5400005e5400005e5400005e540000b0
:100088005e5400005e5400005e5400005e540000a0
:100098005e5400005e5400005e5400005e54000090
:1000a8005e5400005e5400005e5400005e54000080
:1000b8005e5400005e5400005e5400005e54000070
:1000c8005e5400005e5400005e5400005e54000060
:1000d8005e5400005e5400005e5400005e54000050
:1000e8005e5400005e5400005e5400005e54000040
:1000f8005e5400005e5400005e5400005e54000030
:100108005e5400005e5400005e5400005e5400001f
:100118005e5400005e5400005e5400005e5400000f
:100128005e5400005e5400005e5400005e540000ff
:100138005e5400005e5400005e5400005e540000ef
:100148005e5400005e5400005e5400005e540000df
:100158005e5400005e5400005e5400005e540000cf
:100168005e5400005e5400005e5400005e540000bf
:100178005e5400005e540000403d00005e540000e4
:100188005e5400005e5400005e5400005e5400009f
:100198005e5400005e5400005e5400005e5400008f
:1001a8005e5400005e5400005e5400005e5400007f
:1001b8005e5400005e5400005e5400005e5400006f
:1001c8005e5400005e5400005e5400005e5400005f
:1001d8005e5400005e5400005e5400005e5400004f
:1001e8005e5400005e5400005e5400005e5400003f
:0801f8005e5400005e5400009b
:020000040000fa
:100208005e5400005e5400005e5400005e5400001e
:100218005e5400005e5400005e5400005e5400000e
:100228005e5400005e5400005e5400005e540000fe
:100238005e5400005e5400005e5400005e540000ee
:100248005e5400005e5400005e5400005e540000de
:100258005e5400005e5400005e5400005e540000ce
:100268005e5400005e5400005e5400005e540000be
:100278005e5400005e5400005e5400005e540000ae
:100288005e5400005e5400005e5400005e5400009e
:100298005e5400005e5400005e5400005e5400008e
:1002a8005e5400005e5400005e5400005e5400007e
:1002b8005e5400005e5400005e5400005e5400006e
:1002c8005e5400005e5400005e5400005e5400005e
:1002d8005e5400005e5400005e5400005e5400004e
:1002e8005e5400005e5400005e5400005e5400003e
:1002f8005e5400005e5400005e5400005e5400002e
:100308005e5400005e5400005e5400005e5400001d
:100318005e5400005e5400005e5400005e5400000d
:100328005e5400005e5400005e5400005e540000fd
:100338005e5400005e5400005e5400005e540000ed
:100348005e5400005e5400005e5400005e540000dd
:100358005e5400005e5400005e5400005e540000cd
:100368005e5400005e5400005e5400005e540000bd
:100378005e5400005e540000403d00005e540000e2
:100388005e5400005e5400005e5400005e5400009d
:100398005e5400005e5400005e5400005e5400008d
:1003a8005e5400005e5400005e5400005e5400007d
:1003b8005e5400005e5400005e5400005e5400006d
:1003c8005e5400005e5400005e5400005e5400005d
:1003d8005e5400005e5400005e5400005e5400004d
:1003e8005e5400005e5400005e5400005e5400003d
:0803f8005e5400005e54000099
:020000040000fa
:102c5c00486f000073740000202d00002e2d000022
:102c6c002044000065760000202d00002e2d000071
:102c7c00002d00002d2e00002d430000202d000003
:102c8c002d2d00002d2d0000204f0000686d000040
:102c9c0073000000476500006e650000726900005b
:102cac0063200000646500006d6f0000206400006c
:102cbc006576000069630000652000006174000007
:102ccc00746100006368000065640000202d000042
:102cdc00207000006f6c00006c650000642c00001c
:102cec002064000065760000696300006541000007
:102cfc006464000072650000737300003d00000006
:102d0c000d0a0000004400006576000069630000b5
:102d1c006520000066690000726d0000776100009c
:102d2c007265000020760000657200007369000077
:102d3c006f6e0000200000002e00000044650000b3
:102d4c00766900006365000020460000697200008f
:102d5c006d77000061720000652000005665000070
:102d6c0072730000696f00006e2000004572000055
:102d7c00726f0000722100000d0a00000044000078
:102d8c0065760000204600005720000056650000c4
:102d9c007220000045720000726f0000720000008b
:102dac00476500006e65000072690000632000003a
:102dbc00646500006d6f0000206400006576000003
:102dcc006963000065200000646500007461000008
:102ddc006368000065640000202d00002070000076
:102dec006f6c00006c650000640d00000a000000b0
:102dfc003120000044650000766900006365000026
:102e0c002057000072690000746500002045000026
:102e1c00727200006f720000203000007800000019
:102e2c0044650000762000005772000069740000b1
:102e3c006520000045720000726f000072200000d7
:102e4c00003100002044000065760000696300003a
:102e5c006520000052650000616400002045000000
:102e6c00727200006f7200002030000078000000c9
:102e7c00446500007620000052650000616400008b
:102e8c0020450000727200006f72000020200000cc
:102e9c0000320000204400006576000069630000e9
:102eac006520000057720000697400006520000066
:102ebc0045720000726f0000722000003078000034
:102ecc0000320000204400006576000069630000b9
:102edc006520000052650000616400002045000080
:102eec00727200006f720000203000007800000049
:102efc003320000044650000766900006365000023
:102f0c002057000072690000746500002045000025
:102f1c00727200006f720000203000007800000018
:102f2c0033200000446500007669000063650000f2
:102f3c002052000065610000642000004572000012
:102f4c00726f000072200000307800000034000026
:102f5c0020440000657600006963000065200000d5
:102f6c005772000069740000652000004572000073
:102f7c00726f0000722000003078000000340000f6
:102f8c0020440000657600006963000065200000a5
:102f9c005265000061640000204500007272000060
:102fac006f720000203000007800000047650000c0
:102fbc006e6500007269000063200000646500000b
:102fcc006d6f0000206400006576000069630000ee
:102fdc0065200000617400007461000063680000eb
:102fec0065640000202d000020650000766500005f
:102ffc006e7400002c2000006465000076690000ef
:10300c006365000041640000647200006573000099
:10301c00733d000000470000656e00006572000003
:10302c006963000020640000656d00006f200000e3
:10303c006465000076690000636500002064000090
:10304c006574000061630000686500006420000086
:10305c002d20000065760000656e0000740d0000e8
:10306c000a0000000d0a00002a2a00002a2a00008b
:10307c002a20000055530000422000004572000039
:10308c00726f0000722000002d2000006875000097
:10309c00627300002061000072650000206e000069
:1030ac006f7400002073000075700000706f0000da
:1030bc007274000065640000202a00002a2a0000b7
:1030cc002a2a00000d0a0000000d00000a2a000048
:1030dc002a2a00002a2a0000205500005342000032
:1030ec0020450000727200006f720000202d00005d
:1030fc002064000065760000696300006520000014
:10310c0069730000206e00006f74000020730000d3
:10311c0075700000706f0000727400006564000030
:10312c00202a00002a2a00002a2a00000d0a00008a
:10313c00000d00000a2a00002a2a00002a2a00009a
:10314c002055000053420000204500007272000020
:10315c006f720000202d000020630000616e0000e3
:10316c006e6f000074200000656e0000756d00002d
:10317c006572000061740000652000006465000049
:10318c007669000063650000202a00002a2a0000ee
:10319c002a2a00000d0a0000000d00000a2a000077
:1031ac002a2a00002a2a0000205500005342000061
:1031bc0020450000727200006f720000202d00008c
:1031cc00206300006c690000656e00007420000034
:1031dc0064720000697600006572000020690000ce
:1031ec006e69000074690000616c0000697a00006f
:1031fc0061740000696f00006e20000065720000b1
:10320c00726f0000722000002a2a00002a2a000097
:10321c002a0d00000a0000000d0a00002a2a0000f6
:10322c002a2a00002a2000005553000042200000ea
:10323c0045720000726f0000722000002d2000000b
:10324c006f750000742000006f660000206800009d
:10325c0065610000702000006d6500006d6f00005e
:10326c0072790000202a00002a2a00002a2a000075
:10327c000d0a0000000d00000a2a00002a2a000096
:10328c002a2a00002055000053420000204500006f
:10329c00727200006f720000202d0000207500007b
:1032ac006e730000706500006369000066690000c1
:1032bc0065640000202a00002a2a00002a2a000047
:1032cc000d0a0000000d00000a0d00000a4300006a
:1032dc006f7500006c640000206e00006f740000bd
:1032ec00206900006e69000074690000616c0000c8
:1032fc00697a000065200000555300004220000050
:10330c0043750000737400006f6d000020440000d2
:10331c00656d00006f2000004170000070200000ff
:10332c002d2000007379000073740000656d00009f
:10333c002e20000020480000616c00007469000021
:10334c006e6700002e0d00000a0d00000a00000040
:10335c000d0a00000d0a00002a2a00002a2a00008b
:10336c002a20000055530000422000004375000045
:10337c00737400006f6d000020440000656d000048
:10338c006f2000004170000070200000496e0000aa
:10339c0069740000696100006c6900007a650000c6
:1033ac00642000002a2a00002a2a00002a0d0000ae
:1033bc000a0d00000a0000000d0a00000d0a0000b2
:1033cc00436f0000756c0000642000006e6f0000fd
:1033dc0074200000696e00006974000069610000cf
:1033ec006c6900007a650000205500005342000013
:1033fc002043000075730000746f00006d20000006
:10340c00446500006d6f00002041000070700000ea
:10341c00202d000020550000534200002e200000fb
:10342c0020480000616c0000746900006e670000a9
:10343c002e0d00000a0d00000a00000030310000c3
:10344c0032330000343500003637000038390000c4
:0c345c00414200004344000045460000cf
:020000040000fa
:103468000600fa0020479800314798005181200053
:10347800914078002e40900080cf50000300320029
:1034880060002000200798001900370010468000cf
:10349800000f7800120037001e007800c058900016
:1034a8003e40900080cf50000b003a009e0078000c
:1034b800214090000030a100a04098009e007800b4
:1034c800214090000040a100a04098000000eb00bf
:1034d80020079800060037001e007800100f7800bb
:1034e8001e00e000ecff3a00400120002007980091
:1034f8002e0090000080fa00000006001000fa007c
:10350800004f780011479800224798002307980039
:10351800340798004507980056079800474f9800c9
:1035280015c8bf009e4f5000030032006000200005
:1035380070079800530037009142800000f0200087
:103548008080600000402000808f5000030032001f
:1035580011002000710798004a00370010468000cb
:10356800a040900000c8b30000c060000004e00064
:1035780003003a000001200070079800410037005e
:103588002e409000eb4f500002003a000040eb0044
:10359800381007002e409000e14f500005003a0017
:1035a8002e0090000000e00002003a003e0090006b
:1035b80030100700204680009e40900001487800a7
:1035c800204680000000e800ae40900001487800e6
:1035d800204680008080e8002e0090008048780017
:1035e80020468000e30040002e0090004800de00e6
:1035f8008048780020468000e40040003e009000ab
:103608008048780020468000e50040003e00900099
:103618004800de008048780020468000e600400030
:103628004e0090008048780020468000e700400067
:103638004e0090004800de00804878004e48900018
:103648000004e00007003a00214680001046800090
:103658004e029000de01900082002000530d07000a
:103668000600370021468000104680004e02900078
:10367800de019000820020000e0d07000000eb0024
:10368800700798007e0090000080fa000000060095
:103698000400fa00004f78009042800001f02000fa
:1036a800010060000000e00003003a001003200061
:1036b800100798001d0037009142800000f020009c
:1036c8008080600000402000808f50000b003a008e
:1036d80090428000010f200001006000f00f5000b0
:1036e80003003a00a0032000100798000f003700dd
:1036f80000032000100798000c003700914280005a
:1037080000f020008080600000502000808f500072
:1037180004003a0016c8bf000080fb00100798009c
:103728000200370020032000100798001e009000b8
:103738000080fa00000006000600fa00008fbe00b4
:10374800104680000000e0000d003a002002200032
:1037580074fc070010468800104680000000e00056
:1037680003003a000000eb0020079800180037001b
:10377800114680000000eb00800878000100370047
:10378800ac0c070010468000304088000000eb00b9
:10379800904288000080eb00a04288000040eb00c7
:1037a80014e8b7000040eb0015e8b7005608a80079
:1037b80040002000e040880040002000f0408800e1
:1037c8000000eb000041880010002000200798004e
:1037d8002e0090000080fa00000006000c00fa009d
:1037e800204798003147980022079800340798002e
:1037f8004507980051812000914078002e409000a4
:1038080080cf50000300320060002000500798006d
:10381800470037009142800000f02000808060005f
:1038280000402000808f500003003200100020006c
:10383800500798003e00370010468000000f7800bf
:10384800370037001e007800c05890003e409000b6
:1038580080cf500030003a001e007800e008900049
:1038680000302000008060000000e00003003a0003
:1038780080012000500798002d0037001e007800b6
:10388800405890000004e00003003500500120007b
:1038980050079800260037001e007800204090004e
:1038a800684060000004e0000300320010012000be
:1038b800500798001e0037001e0078002040900036
:1038c800704060000004e000030032002001200086
:1038d80050079800160037001e007800a04090009e
:1038e80000c8b30000c060000004e00003003a0014
:1038f80000012000500798000d0037003e0190009d
:10390800ae0090001e007800ed0c07000000eb00f0
:1039180050079800060037001e007800100f780046
:103928001e00e000c7ff3a00400120005007980041
:103938005e0090000080fa00000006000400fa0013
:10394800004f780015c8bf009e4f5000030032009a
:1039580060002000100798000c003700904280009b
:1039680001f02000010060000000e00003003a00c0
:103978003000200010079800040037000000eb001a
:10398800904288000000eb00100798001e0090008d
:103998000080fa00000006000400fa00004f7800da
:1039a80015c8bf009e4f5000030032006000200081
:1039b800100798000c003700914280000041200059
:1039c800808f50000300320030002000100798005c
:1039d80005003700904280000000e800904288000f
:1039e8000000eb00100798001e0090000080fa000d
:1039f800000006000400fa00004f78001147980004
:103a080015c8bf009e4f5000030032006000200020
:103a180010079800150037009142800000f0200040
:103a28008080600000402000808f5000030032003a
:103a380010002000100798000c003700f80f07004e
:103a48000000e0000300320020002000100798006a
:103a5800060037001e40900012e8b700003320002f
:103a6800904288000000eb00100798001e009000ac
:103a78000080fa00000006000200fa000000eb00d7
:103a88004024880015c8bf000004e0000d00320083
:103a98000040eb00004f780015c8bf00240020004c
:103aa800050020000e017800e1002000ba1607008a
:103ab80015c8bf00130020005281200071002000ab
:103ac800070d07006000b8001bff07000080fa0020
:103ad800000006000400fa00004f780015c8bf0077
:103ae8009e4f50000300320060002000100798002d
:103af8000c0037009142800000402000808f500069
:103b0800030032003000200010079800050037003d
:103b18009404a90000412000904288000000eb00b6
:103b2800100798001e0090000080fa0000000600b0
:103b38003200fa00881f780031003700f04080001a
:103b4800e20f500007003c00f04080006c00b90014
:103b580080007800e082200080804000011f9800eb
:103b68000200370020822000001f98008e18900065
:103b7800110798001e009000100078007017980038
:103b88007e109000e10f500004003200fe109000fb
:103b9800e18f400001003200070037001e0090004e
:103ba8000081e8001e0090009000780015c8bf0052
:103bb800a3002000ca0c070060248000000f7800d2
:103bc8000000eb0060248800004180000000e9004c
:103bd80000418800f0408000e20f500004003c00e3
:103be800f04080000000e800f04088000200370044
:103bf8000000eb00f04088009e00780061248800f7
:103c0800004180000000e000ccff3a00a0428000a4
:103c1800e10f400004003200a0428000904288007a
:103c28000080eb00a04288009042800001f0200054
:103c3800010060006017980000202000ee1090003e
:103c4800808f50005202320000202000ee109000b9
:103c5800808f500008003e006e1090000000e000c9
:103c68001200320000102000ee109000808f5000eb
:103c7800a60032009a05370000402000ee109000a0
:103c8800808f50000b05320000502000ee1090008d
:103c9800808f50004405320000302000ee10900064
:103ca800808f5000990232008d05370091428000c4
:103cb800000f200080806000511798005e1090006f
:103cc800f00f50005d00320000022000de1090006e
:103cd800808f5000630032005e1090000000e0000a
:103ce800010032007e05370063ff0700114680009f
:103cf8000000eb0080087800114680000000eb000f
:103d08009000980011468000314090000000a0000b
:103d1800b040980011468000214090000070a0003b
:103d2800a04098001146800000042000c0009800c0
:103d3800124680006000b800000998001109980038
:103d4800114680000040eb00c058980011468000e2
:103d58000040eb00805898001146800061089000f0
:103d68000080a1000090a100e008980011468000a2
:103d78000000eb00d008980030c0b30002e8b7009c
:103d88000040eb0012e8b7000040eb0013e8b70072
:103d98000040eb0014e8b7000000eb00d0408800ba
:103da8000000eb0060248800f00f200050248800f9
:103db8000000eb0010248800f00f20000024880089
:103dc8000000eb0080248800f00f20007024880099
:103dd8008cc4a80000a020004800de00c024880091
:103de80080002000a0248800a0002000a0248800d3
:103df80080002000a0248800c00320003024880010
:103e080020012000302588000000eb0040258800b4
:103e18000000eb00b0248800aae4a900a004200058
:103e2800002588009142800000ff2000008060008b
:103e380070004000904288002905370056c8bf002e
:103e4800614060000004e0002505320091428000d6
:103e580000ff200000806000700040009042880051
:103e68001f053700ec0047000040eb008048780051
:103e7800ec00470020c3b300904098006c01470055
:103e88002400200005002000d100200000c0eb0025
:103e9800c11507000000e0001800320010002000e3
:103ea8004024880071048000f0fb2f00008060002f
:103eb8007004880071068000f00f2f0000806000f9
:103ec8007006880071068000006020000080700085
:103ed80070068800f1048000000420000080700053
:103ee800f00488009142800000ff200000806000fc
:103ef8007000400090428800f90437005608a90075
:103f08000001200090428800f504370090428000ac
:103f1800010f2000010060004017980000022000f7
:103f2800ce109000808f5000b000320000022000b8
:103f3800ce109000808f500007003e004e10900079
:103f48000000e0000d003200ce109000f08f50000d
:103f580029003200e204370000032000ce10900050
:103f6800808f50002901320000042000ce109000fc
:103f7800808f50007f013200d904370090428000c2
:103f88006f006000301798003e109000e10f50005d
:103f9800d3043200be109000e18f500004003900b5
:103fa8003e109000e20f50000d003200cc043700a4
:103fb80010002000502488008c04a800b00f2000b6
:103fc80020408800000420000024880082c4a80043
:103fd800904280000000e80090428800c00437004a
:103fe8009142800000ff20000080600070004000c7
:103ff80090428800ba043700904280006f00600049
:1040080020179800ae109000e28f50006200320036
:104018002e109000e20f500004003e00ae109000f9
:104028000100e00008003200ad0437002e109000b7
:10403800e30f5000aa043200ae109000e48f500045
:1040480060003200a6043700204680000000e0002f
:10405800040032002046800084fa07000000eb00cc
:1040680020468800800020002efa0700204688009d
:10407800204680000000e00005003a0030c3b3008d
:1040880016e8b700005020009042880094043700da
:104098000040eb0012e8b7000040eb0013e8b7005f
:1040a8000000eb00d040880030c0b30001e8b70042
:1040b800d0002000502588000000eb006025880013
:1040c8000000eb00702588000000eb0080258800c8
:1040d8000000eb00902588000000eb00a025880078
:1040e8000000eb00b02588000000eb00c025880028
:1040f8000000eb00d02588000000eb00e0258800d8
:104108000000eb00f02588000000eb000026880086
:104118000000eb00102688000000eb002026880035
:104128000000eb00302688000000eb0040268800e5
:10413800414920009140780000c8b30000c06000e9
:104148000004e00006003a001a08a80000c8b300fe
:1041580014e8b70000082000b0248800aae4a800ea
:104168009424a8009424a9001a88a9001aa8a900d0
:104178009484a80030032000204088000004200018
:104188000024880082c4a800904280000000e80053
:1041980090428800520437009484a9009404a8002f
:1041a800b00020002040880000042000002488007f
:1041b80082c4a800904280000000e8009042880075
:1041c80047043700f000200060248800f00f20002a
:1041d800802488009142800000ff20000080600059
:1041e80070004000904288003d04370090428000f3
:1041f8006f006000101798001e109000e10f50002b
:10420800390032009e109000e18f50000400390000
:104218001e109000e20f50004e00320030043700ac
:10422800004680000000e0000400320000468000e4
:104238000efa07000000eb000046880021468000c7
:1042480000c8b30080487800204680008000e8005d
:1042580060c0b30080487800204680008080e80075
:104268000040eb008048780020468000e3004000d2
:1042780010c0b3008048780020468000e400400069
:104288000040eb008048780020468000e5004000b0
:104298000040eb008048780020468000e60040009f
:1042a80080c0b3008048780020468000e7004000c6
:1042b8000040eb00804878002046800021468000be
:1042c80015468000840020008001780082002000cc
:1042d80005007800f7090700904280000000e80018
:1042e80090428800fe03370010468000a0409000ee
:1042f80000c8b30000c060000004e000f80332000a
:1043080010468000204090000044b2000004e00005
:104318000e00320020468000640040001040780003
:10432800e94f500005003a0050c3b30016e8b70043
:104338000050200090428800e90337009042800036
:104348000000e80090428800e5033700d104070028
:10435800e303370020468000104078000080fb000f
:1043680070f9070000468800004680000000e00061
:1043780005003a0030c3b30016e8b700005020002b
:1043880090428800d603370001468000204680000e
:104398001040780080487800114680002046800050
:1043a800704090000080fb00c0009800204680000c
:1043b800aef907000000eb00204688001046800098
:1043c8004000900057f907002046880020468000ea
:1043d8000000e00005003a0030c3b30016e8b7005b
:1043e8000050200090428800bd03370030c0b30061
:1043f80001e8b7009142800000ff200000806000c3
:104408007000400090428800b50337009042800059
:104418006f006000001798008e109000e18f500028
:104428003b0032000e109000e10f500004003900ec
:104438008e109000e28f500046003200a80337002b
:1044480094c4bf000042b2000004e000a4033a0094
:104458002146800000c8b3008048780020468000cc
:104468008000e80060c0b3008048780020468000e3
:104478008080e8000040eb008048780020468000fb
:10448800e300400010c0b300804878002046800058
:10449800e40040000040eb0080487800204680009f
:1044a800e50040000040eb0080487800204680008e
:1044b800e600400000468000104078008048780000
:1044c80020468000e70040000040eb00804878006c
:1044d80000468000104078000080fb000146800004
:1044e8002546800016468000000278008101780089
:1044f8008200200085007800060078006d0907001a
:10450800904280000000e800904288007403370061
:1045180010468000a040900000c8b30000c06000b2
:104528000004e0006e033200104680002040900036
:104538000044b2000004e000040032009042800011
:104548000000e80090428800650337005104070026
:104558006303370030c0b30001e8b7009142800020
:1045680000ff20000080600070004000904288003a
:104578005b033700a80407009142800000f0200088
:10458800008060000010b00090428800540337009b
:1045980090428000010f2000010060000000e00050
:1045a800010032004e033700904280006f00600027
:1045b800700f98007e089000e10f50003200320022
:1045c800fe089000e18f5000040039007e0890003a
:1045d800e20f50003d0032004103370010c0b30025
:1045e80015e8b700214680000040eb0080487800bd
:1045f800204680008000e80050c0b3008048780062
:10460800204680008080e80015c8bf0080487800f8
:1046180020468000e30040000040eb00804878001e
:1046280020468000e40040000040eb00804878000d
:1046380020468000e50040000040eb0080487800fc
:1046480020468000e60040000040eb0080487800eb
:1046580020468000e70040000040eb0080487800da
:1046680021468000104680000002eb008001eb002c
:10467800820020004d090700904280000000e800f9
:10468800904288001603370010468000a040900032
:1046980000c8b30000c060000004e000100332004e
:1046a80010468000204090000044b2000004e00062
:1046b80004003200904280000000e8009042880028
:1046c80007033700f3030700050337001ac8bf00c4
:1046d800614060000080fb004700dd0080407800fa
:1046e80015c8bf0000c0700014e8b70030c0b300a0
:1046f80001e8b7009142800000f0200000806000cf
:104708000010b00090428800f50237009042800007
:10471800010f200001006000600f980000022000d7
:10472800ee089000808f5000c40032000002200084
:10473800ee089000808f500007003e006e08900041
:104748000000e0000d003200ee089000f08f5000ed
:1047580021003200e202370000032000ee0890003a
:10476800808f50002201320000042000ee089000e3
:10477800808f5000bc013200d9023700004680000b
:104788001050900000e8b7000a003700e0458000ac
:104798001000900030079800e04580001000780075
:1047a800b2f80700e0458000b0f807003e0090002e
:1047b800e0458800e04580000000e000f3ff3a0093
:1047c8009142800000ff20000080600070004000df
:1047d80090428800c2023700904280006f0060005b
:1047e800500f98005e089000e10f5000330032002f
:1047f800de089000e18f5000040039005e08900048
:10480800e20f50003e003200b5023700214680001a
:1048180000c8b30080487800204680008000e80087
:1048280060c0b30080487800204680008080e8009f
:1048380000c8bf000040e90080487800204680009a
:10484800e300400020c0b300804878002046800084
:10485800e40040000040eb008048780020468000db
:10486800e50040000040eb008048780020468000ca
:10487800e600400080c0b3008048780020468000f1
:10488800e70040000040eb008048780020468000a8
:1048980021468000154680008400200080017800b1
:1048a80082002000050078008208070090428000fe
:1048b8000000e80090428800890237001046800016
:1048c800a040900000c8b30000c060000004e000f1
:1048d8008302320010468000204090000044b2005d
:1048e8000004e00004003200904280000000e8006c
:1048f800904288007a023700660307007802370082
:104908006000200007f80700300798003e0090007c
:104918000000e00005003a0030c3b30016e8b70015
:1049280000502000904288006d0237003e0490003d
:104938002046800063004000104078000080fb00a3
:10494800c800dd00204680000080e80010407800a4
:104958000080fb0000804000f2f70700000c7800a0
:10496800180078000000e00009003a003e009000be
:104978003ef807000000eb003007980030c3b30092
:1049880016e8b70000502000904288005402370013
:104998003e0090001000780000017800204680005a
:1049a80063004000104078000080fb00c800dd0074
:1049b800204680000080e800104078000080fb005e
:1049c80080814000f00f200080806100224090002c
:1049d800604060000140700020419800c818de0067
:1049e8003240900060406000014070003041980003
:1049f800be009000e0458000900098003e009000c6
:104a0800e04588003e00900010007800f0458800de
:104a1800be00900000c8bf00c040980030c0b3007e
:104a280001e8b7009142800000ff2000008060008c
:104a380070004000904288002902370090428000b0
:104a48006f006000400f9800ce089000e18f500082
:104a5800450032004e089000e10f50000400390074
:104a6800ce089000e28f5000500032001c02370040
:104a78002146800000c8b3008048780020468000a6
:104a88008000e80060c0b3008048780020468000bd
:104a98008080e80000c8bf000040e9008048780036
:104aa80020468000e300400020c0b3008048780022
:104ab80020468000e40040000040eb008048780079
:104ac80020468000e50040000040eb008048780068
:104ad80020468000e6004000e04580001000780095
:104ae8000080e80010407800804878002046800068
:104af800e7004000e04580001000780063004000b7
:104b08001040780080487800e04580001000780068
:104b180080007800214090000081fb003140900027
:104b28000080fb004800dd00020070008000780073
:104b3800e045800010007800254680001646800079
:104b4800010278008001780082002000850078004a
:104b580006007800d7070700904280000000e800b0
:104b680090428800de01370010468000a040900087
:104b780000c8b30000c060000004e000d8013200a3
:104b880010468000204090000044b2000004e0007d
:104b980004003200904280000000e8009042880043
:104ba800cf013700bb020700cd01370030c0b3008a
:104bb80001e8b70000c8bf000040e90000e8b700fe
:104bc80000c8bf000004e0000300320000312000ec
:104bd80090428800c20137009142800000ff200007
:104be800008060007000400090428800bc013700df
:104bf800904280006f006000300f98003e089000df
:104c0800e10f500042003200be089000e18f5000d2
:104c1800070039003e089000e20f5000790032008a
:104c2800be089000e38f500087003200ac013700c7
:104c38005b07070012c8bf000004e00011003a003b
:104c4800e0458000500798000a0037005e00900099
:104c580010007800f0458800fd0807000000e0001b
:104c68001f003a004e0707005e0090009000900079
:104c7800510798005e0090000000e000f3ff3a0042
:104c880017003700e0458000500798000300370000
:104c98005e00900090009000510798005e00900020
:104ca8000000e000050032005e009000c040900067
:104cb80012c8bf0080cf5000f5ff3a005e00900098
:104cc80010007800f0458800e10807000000e000c7
:104cd80003003a00320707000000eb005007980075
:104ce8005e0090000000e00005003a0040c3b300f9
:104cf80016e8b7000050200090428800780137007d
:104d0800904280000000e80090428800740137005b
:104d18001ac8bf00644060000004e00033003a0095
:104d28001a48a800214680000040eb00804878001f
:104d3800204680008000e80030c0b300804878003a
:104d48001ac8bf00684060000004e0000500320097
:104d5800204680008080e80030c0b300804878009a
:104d680004003700204680008080e80040c0b3007f
:104d78008048780020468000e30040000040eb00b7
:104d88008048780020468000e40040000040eb00a6
:104d98008048780020468000e50040000040eb0095
:104da8008048780020468000e60040000040eb0084
:104db8008048780020468000e70040000040eb0073
:104dc8008048780021468000104680000002eb00f1
:104dd8008001eb00820020007407070090428000e9
:104de8000000e800904288003d01370091428000b1
:104df80000ff2000008060007000400090428800a2
:104e08003701370010468000a040900000c8b3006a
:104e180000c060000004e00031013200104680004c
:104e2800204090000044b2000004e000040032007a
:104e3800904280000000e800904288002801370076
:104e4800140207002601370030c0b30001e8b7009c
:104e58009142800000ff2000008060007000400048
:104e6800904288001e013700904280006f00600069
:104e7800200f98002e089000e10f500033003200f8
:104e8800ae089000e18f5000070039002e0890000e
:104e9800e20f50003e003200ae089000e38f500051
:104ea800410032000e013700214680000040eb002f
:104eb80080487800204680008000e80090c0b30059
:104ec80080487800204680008080e80012c8bf0033
:104ed8008048780020468000e30040000040eb0056
:104ee8008048780020468000e40040000040eb0045
:104ef8008048780020468000e50040000040eb0034
:104f08008048780020468000e60040000040eb0022
:104f18008048780020468000e70040000040eb0011
:104f28008048780021468000104680000002eb008f
:104f38008001eb00820020001c07070090428000df
:104f48000000e80090428800e50037001046800025
:104f5800a040900000c8b30000c060000004e0005a
:104f6800df00320010468000204090000044b2006c
:104f78000004e00004003200904280000000e800d5
:104f880090428800d6003700c2010700d4003700dd
:104f980030c0b30001e8b700904280000000e8008c
:104fa80090428800ce0037009142800000f0200037
:104fb800008060000010b000904288001ac8bf004e
:104fc8000044b2000004e0001800320017c8bf0017
:104fd800404798004e4090000080fb00c300dd0071
:104fe800c08a200000804000100278004e409000e7
:104ff8000080fb004300dd00e4004000c08a200080
:10500800008040001001be0015c8bf000400010068
:105018000000e000b2003a0090c3b30016e8b70001
:105028000050200090428800ad00370031468000d3
:10503800410798001b0037004e009000c0409000c8
:10504800414798004e4090000080fb00c300dd00ff
:10505800c08a200000804000100278004e40900076
:105068000080fb004300dd00e4004000c08a20000f
:10507800008040001001be0015c8bf0004000100f8
:105088000000e00004003a0090c3b30016e8b7003f
:1050980000502000904288004e0090009000780058
:1050a800410798004e0090000000e000e2ff3a003f
:1050b8008b00370091428000000f20008080600044
:1050c800110f98001e0890000000e00084003200d4
:1050d8009e089000f08f50000100320080003700d9
:1050e800904280006f006000000f98000e0890004a
:1050f800e20f50007a0032008e089000e28f5000d4
:1051080007003e000e0890000000e0007400320026
:105118008e089000e18f50000b00320070003700bd
:105128000e089000e40f50006d0032008e089000c9
:10513800e48f50000e0039000e089000e50f500073
:1051480016003200660037009444a8005001200081
:1051580020408800000420000024880082c4a800a1
:10516800904280000000e800904288005c00370010
:105178009444a9009404a800b000200020408800ae
:10518800000420000024880082c4a8009042800007
:105198000000e800904288005100370000402000dd
:1051a800904288004e00370090428000010f200096
:1051b800010060000000e0000100320048003700f4
:1051c80080002000a02488000000eb0060248800f4
:1051d800f00f2000502488000000eb001024880005
:1051e800f00f2000002488000000eb0080248800d5
:1051f800f00f2000702488008c04a80016c8bf0097
:105208000080fb007007980040032000fe0090001b
:10521800808f50001800320040032000fe009000ec
:10522800808f500008003c007e009000e70f50007f
:105238001400320030032000fe009000808f5000e0
:10524800160032001800370050032000fe009000be
:10525800808f50000500320090032000fe0090006f
:10526800808f50000a0032000f00370080c0b30062
:10527800404798000e00370000c1b300404798002f
:105288000b00370010c1b3004047980008003700f2
:1052980020c1b300404798000500370030c1b30073
:1052a800404798000200370040c1b30040479800cb
:1052b8004e4090008080fb0015c8bf0014002000fd
:1052c8000500200082812000b31007009142800071
:1052d80000ff2000008060007000400090428800bd
:1052e8004f0478000080fa00000006000400fa006d
:1052f800204798003147980051812000914078005c
:105308002e40900080cf500015003a0010468000d3
:10531800000f7800100037001e007800c058900079
:105328003e40900080cf500009003a009e0078006f
:10533800214090000050a000a04098009e007800f6
:10534800214090000070a000a040980004003700a1
:105358001e007800100f78001e00e000eeff3a00f3
:105368000080fa00000006000c00fa004047980090
:105378005147980032079800430798005181200050
:10538800914078004e40900080cf500009003200d4
:10539800be00900060c0b300804878004e019000c5
:1053a8006000b8000089be00100020005007980077
:1053b8003f0037001146800011079800340037007d
:1053c8001e009000c05890005e40900080cf5000b2
:1053d8002c003a001e009000204090000080fb0046
:1053e8004700de00004f78001e009000204090002b
:1053f8000044b2000004e00009003200be00900042
:105408000040eb00804878001e0090009008900053
:10541800000890004e0190000089be001600370079
:105428001e00900020409000684060000004e000ea
:1054380004003200be00900010c1b300804878001c
:105448000d0037001e009000204090007040600062
:105458000004e000050032001e009000e0589000b3
:105468003e0090000148780003003700be0090001d
:1054780090c1b300804878001e80fb005007980058
:105488000b0037001e00900090007800110798006c
:105498001e0090000000e000c9ff3a00be00900026
:1054a80040c1b300804878001000200050079800e1
:1054b8005e0090000080fa00000006000600fa0076
:1054c800000f780021479800324798002e4090003e
:1054d800e14f400012003a003e4090000004e00016
:1054e8000f003a00c00020009e0f100005003a008f
:1054f80061f907005608a9000000eb002007980092
:1055080009003700f00020009e0f100004003a0048
:105518005608a8000000eb0020079800020037009a
:1055280030002000200798002e0090000080fa002c
:10553800000006000c00fa00204798003147980048
:1055480022079800340798004507980051812000e9
:10555800914078002e40900080cf50000300320028
:1055680060002000500798004700370091428000f3
:1055780000f020008080600000402000808f5000f4
:105588000300320010002000500798003e0037004a
:1055980010468000000f7800370037001e007800a2
:1055a800c05890003e40900080cf500030003a0034
:1055b8001e007800e00890000030200000806000a5
:1055c8000000e00003003a00800120005007980026
:1055d8002d0037001e007800405890000004e000bd
:1055e80003003d00500120005007980026003700b6
:1055f8001e00780020409000684060000004e00031
:105608000300320010012000500798001e003700e8
:105618001e00780020409000704060000004e00008
:1056280003003200200120005007980016003700c0
:105638001e007800a040900000c8b30000c06000c1
:105648000004e00003003a00000120005007980021
:105658000d0037003e019000ae0090001e0078005b
:10566800db0507000000eb00500798000600370034
:105678001e007800100f78001e00e000c7ff3a00f7
:1056880040012000500798005e0090000080fa005a
:10569800000006000000fa00314080002140900020
:1056a8000040a100a04098003140800021409000b7
:1056b8000030a100a040980001c8bf000040e900e8
:1056c80001e8b70001c8bf000004e000050032008f
:1056d8009042800001ff2f00010060009042880086
:1056e8000d00370002c8bf000040e90002e8b7001b
:1056f80002c8bf000004e0000300320000112000cf
:10570800904288000400370070c0b30016e8b70064
:1057180000502000904288000080fa000000060037
:105728000a00fa002047980031479800424798003d
:10573800330798000000eb00000f78002f003700b7
:105748001e0078004300dd00e6004000408b20008a
:1057580000804000100078000000d1006140600027
:10576800e14f500024003a001e007800c300dd001d
:10577800408b200000804000904078002e40900030
:1057880080cf50001c003a001e007800c300dd00e6
:10579800408b200000804000904090003e409000e8
:1057a80080cf500014003a001e0078004300dd004e
:1057b8008080e800408b2000008040009040780006
:1057c8004e40900080cf50000b003a001e00780039
:1057d8004300dd00e4004000408b200000804000d2
:1057e800904090003e009000014878001000200092
:1057f80040079800050037001e0fe8001e00e00073
:10580800cfff34000000eb00400798004e009000e6
:105818000080fa00000006000600fa00004680003a
:10582800000f78000000eb00100798001ac8a900c4
:10583800680037001e0090004300dd00e6004000cd
:10584800408b200000804000100078000000d1004c
:10585800614060000004e0001e0032001e0090005d
:10586800c300dd00408b200000804000904078009d
:105878001e0078004040900080cf500033003a006e
:105888001e009000c300dd00408b20000080400017
:10589800904090001e0078005040900080cf50004b
:1058a8002a003a001e0090004300dd008080e800d6
:1058b800408b200000804000904078001e00780057
:1058c8006040900080cf500020003a001ac8a8001d
:1058d8001e0037001e009000c300dd00408b200032
:1058e80000804000900178009e00780001489000f8
:1058f8000081fb00114890000080fb004800dd009b
:1059080002007000808f510010003a001e009000c5
:105918004300dd008080e800408b200000804000cc
:10592800900178009e007800214890000081fb00db
:10593800314890000080fb004800dd000200700044
:10594800808f510001003a001ac8a8001ac8bf0089
:105958000044b2000004e0001b0032001e0090006a
:105968004300dd00e4004000408b20000080400040
:105978001040900017e8b7001e0090004300dd00bb
:10598800e6004000408b20000080400010007800b6
:105998004200de00614060000004e00007003200c1
:1059a8001e0090004300dd00e4004000408b200012
:1059b800008040001040780012e8b7001000200076
:1059c80020079800080037001e0090000000e8003b
:1059d800100798001e0090000000e00095ff3200bc
:1059e8000000eb00200798002e0090000080fa00cd
:1059f800000006000600fa0020479800314798008a
:105a080030468000000f78000d0037001e00780037
:105a1800a04090002e40900080cf500008003a002f
:105a28001e007800b04090003e40900080cf5000ab
:105a380003003a001e007800200798000400370091
:105a48001e00e000f1ff3a000000eb00200798007c
:105a58002e0090000080fa00000006002800fa00de
:105a68000000eb00200f98009042800094c4bf0013
:105a78000042b2000004e000c7033a008080200022
:105a880010407800614060000004e0005c023a00c9
:105a980010468000300f9800520237003e089000f0
:105aa800e008900000302000008060000000e00066
:105ab80049023a003e089000a040900000c8b30098
:105ac80000c060000004e00043023a003e08900075
:105ad800304088003e089000005890008080fb000d
:105ae800000f20008080600031179800000220001d
:105af800be109000808f5000b500320000032000d7
:105b0800be109000808f50006c0132003e10900053
:105b1800f00f500001003200230237003e089000c9
:105b2800005890000080fb006f006000201798006c
:105b3800ae109000e18f50001d0032002e10900032
:105b4800e10f500004003c00ae1090000100e0009e
:105b5800080032009b0037002e109000e20f500022
:105b680028003200ae109000ef8f50005e00320027
:105b78009400370031408000314090000010a100af
:105b8800b0409800d0c0b300fb0607003e08900064
:105b980040589000d1c0b300cd0607008180200096
:105ba800114078000000a000804878007a03370090
:105bb800324080003040800090089000000890003b
:105bc80050019800610198003140800031409000f8
:105bd8000010a000b040980090c0b300e60607008f
:105be8003e0890004058900091c0b300b8060700e6
:105bf80081802000114078000000a00080487800d3
:105c080065033700be0890000040eb0080589800fc
:105c1800be089000214090000070a000a0409800ad
:105c280000418000e30f50002b003c000041800041
:105c38000000e80000418800e0408000e20f5000ca
:105c480004003c00e04080000000e800e0408800dc
:105c5800020037000000eb00e0408800e0408000d0
:105c68006c00b9008000780020822000008040008d
:105c7800100f98009e0890001000200080087800ff
:105c88003e08900090089000000890001e099000bf
:105c980010019800210198003e089000b00890007b
:105ca8001e089000310098003e089000c0589000ef
:105cb8001e089000014898009e0890000040eb00e4
:105cc800904898003e089000d05890001e08900018
:105cd80021489800b6013700be08900080c0b30084
:105ce800d0589800b2013700be0890000040eb0081
:105cf80080589800be089000214090000070a000d5
:105d0800a040980000418000e30f500029003c00ab
:105d1800004180000000e80000418800e040800069
:105d2800e20f500004003c00e04080000000e80062
:105d3800e0408800020037000000eb00e0408800e7
:105d4800e04080006c00b9008000780020822000cc
:105d580000804000000f98008e0890000080eb0043
:105d6800800878000e0990006000b80010019800c3
:105d7800210198008e0890000000eb00b000980008
:105d88003e089000c05890000e0890000148980006
:105d98003e089000e05890000e08900011489800c6
:105da8003e089000d05890000e08900021489800b6
:105db8007f013700be08900080c0b300d05898001b
:105dc8007b01370010002000200f98007801370071
:105dd8003e089000005890000080fb006f006000b3
:105de800101798001e109000e20f50002b00320090
:105df8009e109000e28f500007003c001e1090009b
:105e08000000e0000b0032009e109000e18f50006f
:105e180017003200a60037001e109000e30f500054
:105e2800330032009e109000ef8f5000690032005e
:105e38009f00370031408000314090000010a100e1
:105e4800b0409800d0c0b3004b0607003e08900051
:105e580040589000d1c0b3001d0607008180200083
:105e6800114078000000a00080487800ca0237007e
:105e780090c0b300400607003e08900040589000cc
:105e880091c0b300120607008180200011407800fd
:105e98000000a00080487800bf0237003240800030
:105ea8003040800090089000000890005001980051
:105eb8006101980031408000314090000010a0003e
:105ec800b040980010c0b3002b0607003e089000b1
:105ed8004058900011c0b300fd05070081802000e4
:105ee800114078000000a00080487800aa0237001e
:105ef800be0890000040eb0080589800be08900053
:105f0800214090000070a000a0409800004180004f
:105f1800e30f50002b003c00004180000000e80027
:105f280000418800e0408000e20f500004003c007f
:105f3800e04080000000e800e040880002003700f0
:105f48000000eb00e0408800e04080006c00b900f1
:105f580080007800208220000080400070079800b0
:105f6800fe00900010002000800878003e08900095
:105f780090089000000890007e01900010019800a1
:105f8800210198003e089000b00890007e00900023
:105f9800310098003e089000c05890007e009000a4
:105fa80001489800fe0090000040eb0090489800df
:105fb8003e089000d05890007e009000214898003c
:105fc800fb003700be08900080c0b300d05898008e
:105fd800f7003700be0890000040eb00805898009a
:105fe800be089000214090000070a000a0409800da
:105ff80000418000e30f500029003c000041800070
:106008000000e80000418800e0408000e20f5000f6
:1060180004003c00e04080000000e800e040880008
:10602800020037000000eb00e0408800e0408000fc
:106038006c00b900800078002082200000804000b9
:1060480060079800ee0090000080eb008008780060
:106058006e0190006000b8001001980021019800be
:10606800ee0090000000eb00b00098003e089000a1
:10607800c05890006e009000014898003e089000bb
:10608800e05890006e009000114898003e0890007b
:10609800d05890006e00900021489800c400370046
:1060a800be08900080c0b300d0589800c0003700e8
:1060b80010002000200f9800bd0037003e08900017
:1060c800005890000080fb006f00600000179800e7
:1060d8000e109000e20f50002b0032008e1090003e
:1060e800e28f500007003c000e1090000000e00016
:1060f8000b0032008e109000e18f50001700320024
:10610800a60037000e109000e30f50003300320055
:106118008e109000ef8f5000690032009f0037000a
:1061280031408000314090000010a100b04098003c
:10613800d0c0b300900507003e089000405890007a
:10614800d1c0b300620507008180200011407800ab
:106158000000a000804878000f02370010c0b3008c
:10616800850507003e0890004058900011c0b30014
:106178005705070081802000114078000000a0002a
:1061880080487800040237003240800030408000a8
:106198009008900000089000500198006101980054
:1061a80031408000314090000010a000b0409800bd
:1061b80090c0b300700507003e089000405890005a
:1061c80091c0b3004205070081802000114078008b
:1061d8000000a00080487800ef013700be0890005a
:1061e8000040eb0080589800be08900021409000c5
:1061f8000070a000a040980000418000e30f50000c
:106208002b003c00004180000000e80000418800ad
:10621800e0408000e20f500004003c00e0408000b5
:106228000000e800e0408800020037000000eb00b2
:10623800e0408800e04080006c00b90080007800f1
:10624800208220000080400050079800de00900067
:1062580010002000800878003e0890009008900008
:10626800000890005e01900010019800210198003c
:106278003e089000b00890005e0090003100980041
:106288003e089000c05890005e00900001489800b9
:10629800de0090000040eb00904898003e08900017
:1062a800d05890005e0090002148980040003700c8
:1062b800be08900080c0b300d05898003c0037005a
:1062c800be0890000040eb0080589800be0890007f
:1062d800214090000070a000a0409800004180007c
:1062e800e30f500029003c00004180000000e80056
:1062f80000418800e0408000e20f500004003c00ac
:10630800e04080000000e800e0408800020037001c
:106318000000eb00e0408800e04080006c00b9001d
:10632800800078002082200000804000400798000c
:10633800ce0090000080eb00800878004e019000ad
:106348006000b8001001980021019800ce0090006c
:106358000000eb00b00098003e089000c058900084
:106368004e009000014898003e089000e0589000c8
:106378004e009000114898003e089000d0589000b8
:106388004e0090002148980009003700be08900090
:1063980080c0b300d05898000500370010002000d6
:1063a800200f98000200370010002000200f9800ee
:1063b8002e0890000000e00007003200be089000a0
:1063c8000040eb0080589800be08900021409000e3
:1063d8000070a000a04098003e089000900078004f
:1063e800310f98003e0890000000e000abfd3a0035
:1063f80081802000114078000000a00080487800cb
:106408008080200010407800684060000004e000b0
:1064180061013a0010468000300f98000040eb0000
:10642800005f98004e0137003e089000e008900099
:10643800003020008080600000202000808f500005
:1064480044013a003e089000a040900000c8b30004
:1064580000c060000004e0003e013a003e089000e1
:1064680030409000644060000004e00039013a00c8
:106478000e5890000040e800005f980080802000df
:10648800e04090000e58900080cf5000310131005c
:106498003e08900030408800808020008e58900090
:1064a800614098003e089000005890008080fb00f2
:1064b800000f200080806000710f98000008200005
:1064c800fe089000808f500005003200000920006f
:1064d800fe089000808f50008a00320011013700ba
:1064e8003e089000005890000080fb006f0060009c
:1064f800600f98006e089000e10f50000e00320007
:10650800ee089000ef8f5000440032006e089000b3
:106518000000e000010032007700370090c0b300af
:10652800950407003e0890004058900091c0b300c1
:106538006704070018013700be0890000040eb0010
:1065480080589800be089000214090000070a0007c
:10655800a040980000418000e30f50002b003c0051
:10656800004180000000e80000418800e040800011
:10657800e20f500004003c00e04080000000e8000a
:10658800e0408800020037000000eb00e04088008f
:10659800e04080006c00b900800078002082200074
:1065a8000080400030079800be00900010002000d6
:1065b800800878003e08900090089000000890003d
:1065c8003e01900010019800210198003e089000bb
:1065d800b00890003e009000310098003e089000fe
:1065e800c05890003e00900001489800be009000fe
:1065f8000040eb00904898003e089000d05890006a
:106608003e00900021489800c8003700be0890005e
:1066180080c0b300d0589800c4003700be0890006e
:106628000040eb0080589800be0890002140900080
:106638000070a000a040980000418000e30f5000c7
:1066480029003c00004180000000e800004188006b
:10665800e0408000e20f500004003c00e040800071
:106668000000e800e0408800020037000000eb006e
:10667800e0408800e04080006c00b90080007800ad
:10668800208220000080400020079800ae00900083
:106698000080eb00800878002e0190006000b800b0
:1066a8001001980021019800ae0090000000eb0056
:1066b800b00098003e089000c05890002e0090004e
:1066c800014898003e089000e05890002e00900085
:1066d800114898003e089000d05890002e00900075
:1066e8002148980091003700be08900080c0b30090
:1066f800d05898008d00370010002000200f980017
:106708008a0037003e089000005890000080fb0087
:106718006f006000500f9800de089000e18f500075
:106728000e0032005e089000ef0f50004400320067
:10673800de0890000100e00001003200760037001a
:1067480010c0b3000c0407003e08900040589000a9
:1067580011c0b300de0307008f003700be089000a9
:106768000040eb0080589800be089000214090003f
:106778000070a000a040980000418000e30f500086
:106788002b003c00004180000000e8000041880028
:10679800e0408000e20f500004003c00e040800030
:1067a8000000e800e0408800020037000000eb002d
:1067b800e0408800e04080006c00b900800078006c
:1067c8002082200000804000100798009e00900062
:1067d80010002000800878003e0890009008900083
:1067e800000890001e0190001001980021019800f7
:1067f8003e089000b00890001e00900031009800fc
:106808003e089000c05890001e0090000148980073
:106818009e0090000040eb00904898003e089000d1
:10682800d05890001e009000214898003f00370083
:10683800be08900080c0b300d05898003b003700d5
:10684800be0890000040eb0080589800be089000f9
:10685800214090000070a000a040980000418000f6
:10686800e30f500028003c00004180000000e800d1
:1068780000418800e0408000e20f500004003c0026
:10688800e04080000000e800e04088000200370097
:106898000000eb00e0408800e04080006c00b90098
:1068a8008000780020822000008f40009e00780041
:1068b8000080eb00800878001e0178006000b800b6
:1068c80010019800210198009e0078000000eb005c
:1068d800b00098003e089000c05890001e00780054
:1068e800014898003e089000e05890001e0078008b
:1068f800114898003e089000d05890001e0078007b
:106908002148980009003700be08900080c0b300f5
:10691800d05898000500370010002000200f98007c
:106928000200370010002000200f98002e08900069
:106938000000e00007003200be0890000040eb00b5
:1069480080589800be089000214090000070a00078
:10695800a04098003e08900090007800310f980001
:106968003e0890000000e000affe3a000e5890008c
:106978000004e00004003200818020000040eb00a9
:10698800e04098009efe370081802000114078008a
:106998000030a000804878000080fa00000006005f
:1069a8000200fa0007003700304680001000780027
:1069b800000f7800304680002cf007001e00780099
:1069c80030468800304680000000e000f6ff3a00bc
:1069d800104680000000e000120032000a00370074
:1069e800104680001000780010007800000f780032
:1069f80010468000100078001cf007001146800047
:106a08001e0078008008780010468000100078008a
:106a18000000e000f2ff3a00114680000000eb00a1
:106a28008008780010468000304088000080fa0016
:106a3800000006000200fa000a003700e045800066
:106a480010009000000f7800e045800010007800ea
:106a580006f00700e045800004f007001e007800fb
:106a6800e0458800e04580000000e000f3ff3a00c0
:106a7800004680000000e00004003200004680006c
:106a8800faef07000000eb0000468800204680006f
:106a98000000e0000400320020468000f3ef070009
:106aa8000000eb0020468800bdff07000080fa00c8
:106ab800000006000a00fa00000f7800110798008d
:106ac8002207980033079800440798009e00780032
:106ad800214090000030a100a04098009e0078005e
:106ae800214090000040a100a04098009e0078003e
:106af800214090000050a100a04098009e0078001e
:106b0800214090000060a100a04098009e007800fd
:106b1800214090000000a1000010a1000020a10069
:106b2800a04098009e007800314090000020a1000d
:106b3800b04098001e007800be0090003108980010
:106b48001e0178006000b80000099800110998003b
:106b58004e009000010020001e01780050019800ae
:106b6800610198009e0078000000eb0080109800fa
:106b78001e0078009e009000210898001e007800f2
:106b8800ae009000710098009e00780000c2b3002b
:106b9800805898009e007800214090000070a10065
:106ba800a04098000080fa00000006000a00fa00e1
:106bb800000f780011079800220798003307980003
:106bc800440798009e007800214090000030a10002
:106bd800a04098009e007800214090000040a1004d
:106be800a04098009e007800214090000050a1002d
:106bf800a04098009e007800214090000060a1000d
:106c0800a04098009e007800214090000000a1005c
:106c18000010a1000020a100a04098009e0078006c
:106c2800314090000020a100b04098001e0078007c
:106c3800be009000310898001e0178006000b8007e
:106c480000099800110998004e00900001002000ea
:106c58001e01780050019800610198009e0078009c
:106c68000000eb00801098001e0078009e00900045
:106c7800210898001e007800ae009000710098006e
:106c88004e0090000000e00004003a009e007800ea
:106c980000c1b30080589800030037009e007800b8
:106ca80000c3b300805898009e00780021409000ef
:106cb8000070a100a04098000080fa0000000600c3
:106cc8000600fa00000f78001107980022079800c4
:106cd8009e007800214090000050a100a04098003c
:106ce8009e007800214090000060a100a04098001c
:106cf8009e007800214090000000a1000010a10033
:106d08000020a100a04098009e007800314090002b
:106d18000020a100b04098001e0078009e0090005e
:106d2800310898001e0178006000b800000998003a
:106d3800110998002e009000010020001e01780023
:106d480050019800610198009e0078000000eb0057
:106d5800801098001e007800e008900000302000a5
:106d68008080600000302000808f500004003a00ce
:106d78009e00780000c4b300805898000e003700c9
:106d88001e007800e008900000302000808060003d
:106d980000102000808f500004003a009e00780008
:106da80000c6b30080589800030037009e007800a2
:106db80000c8b300805898009e00780021409000d9
:106dc8000070a100a04098000080fa0000000600b2
:106dd8000600fa00000f78001107980022079800b3
:106de8009e007800214090000050a100a04098002b
:106df8009e007800214090000060a100a04098000b
:106e08009e007800214090000000a1000010a10021
:106e18000020a100a04098009e007800314090001a
:106e28000020a100b04098001e0078009e0090004d
:106e3800310898001e0178006000b8000009980029
:106e4800110998002e009000010020001e01780012
:106e580050019800610198009e0078000000eb0046
:106e6800801098001e007800e00890000030200094
:106e78008080600000302000808f500004003a00bd
:106e88009e00780000c5b300805898000e003700b7
:106e98001e007800e008900000302000808060002c
:106ea80000102000808f500004003a009e007800f7
:106eb80000c7b30080589800030037009e00780090
:106ec80000c9b300805898009e00780021409000c7
:106ed8000070a100a04098000080fa0000000600a1
:106ee8000e00fa00404798003107980042079800c2
:106ef800530798001046800010079800314680001c
:106f0800010f78001ac8bf000044b2000004e00076
:106f18000f00320017c8bf000080fb004300dd00ef
:106f28008080e800c08a200000804000900178003e
:106f38005e009000010020000002be004e0190009b
:106f4800be0090004e409000030001003e00370054
:106f58003e00900060079800ee009000e18f50001e
:106f6800220032006e009000e10f40001f00320046
:106f7800330037001e009000500890000000e00029
:106f8800170032001e009000c05890004e0090007c
:106f98006040900080cf500011003a001e00900021
:106fa80050089000404090000080fb004300dd0046
:106fb8008080e800c08a20000080400090017800ae
:106fc8005e009000010020000002be004e0190000b
:106fd800be0090004e409000030001001a003700e8
:106fe8001e00900090007800110798001e00900085
:106ff8000000e000dfff3a00130037001e007800b1
:10700800404090000080fb004300dd008080e800e5
:10701800c08a200000804000900178005e00900047
:10702800010020000002be004e019000be0090004a
:107038004e409000030001001e007800100f7800f9
:107048001e00e000edff3a000080fa000000060094
:107058001e00fa000000eb0030079800f0458000a1
:10706800000f78000040eb00004f98000040eb0054
:10707800304f98001a28a9001a48a8001e00780066
:1070880090407800415798001e0fe8001e007800d5
:1070980090407800615798001e0fe8001e007800a5
:1070a800104078000080fb00600798001e0fe80081
:1070b8001e007800104078000080fb004800dd00ca
:1070c800800078006e009000010040006007980082
:1070d8001e0fe8001e0078009040780021579800a5
:1070e8001e0fe8001e00780090407800214f98009d
:1070f8001e0fe8001e0fe8001e0fe8001e007800b3
:107108009040780011579800790047009e509000f1
:1071180011409800f90047000040eb0080487800d3
:10712800790147002400200005002000d10020003c
:1071380000c0eb00180907000000e00005003a0055
:1071480080c2b30016e8b7000000eb00600f98009b
:10715800450137004e5090008080fb003e009000b3
:107168000100400030079800f14580003e00900083
:10717800008f40002a0137001e00780090407800f8
:10718800415798001e0fe8001e00780090407800d4
:10719800615798001e0fe8006e509000e94f5000ac
:1071a8000f003a001a28a8001e0078001040780046
:1071b80013e8b70013c8bf000080fb000000d1002f
:1071c800610060000004e000050032001ac8bf003a
:1071d800684060000004e000010032001a48a9007d
:1071e8006e509000e44f5000090032004e5090005d
:1071f8008080fb003e0090000100400030079800ae
:10720800f14580003e009000008f400004013700e7
:107218001e00780090407800515798001e0fe80033
:107228001e00780090407800715798001e0fe80003
:107238001e00780090407800315798001e0fe80033
:107248001e00780090407800015798001e0fe80053
:107258001e00780090407800714f98001e0fe800db
:107268001e00780090407800614f98001e0fe800db
:107278001ac8bf000044b2000004e0000300320056
:1072880017c8bf00005f9800140037007800470057
:10729800800178006e499000fe4890000e509000e2
:1072a8001ff907000000e0000c003a003e4890007b
:1072b8000040e800304f98004e5090008080fb005e
:1072c8003e0090000100400030079800f145800022
:1072d8003e009000008f4000d10037008e4890009b
:1072e8005e50900080cf500004003a00be489000e5
:1072f8007e50900080cf5000090032004e50900020
:107308008080fb003e00900001004000300798009c
:10731800f14580003e009000008f4000c00037001b
:10732800600020007fed0700100798001e00900005
:107338000000e00003003a000000eb00600f980036
:10734800c90037001e009000de50900021409800d0
:107358001e009000fe509000314098008e5890001a
:107368001e00900041409800314680001e009000a9
:10737800010878001e009000304688000e489000f2
:107388000040e800004f98000040eb00304f9800a4
:107398000040eb00104f98004e5090008080fb009a
:1073a8003e0090000100400030079800f145800041
:1073b8003e009000008f40008a0037001e007800d1
:1073c80090407800415798001e0fe8001e00780092
:1073d80090407800615798001e0fe8006e509000aa
:1073e800e54f5000090032004e5090008080fb00ad
:1073f8003e0090000100400030079800f1458000f1
:107408003e009000008f40007600370020022000e8
:1074180044ed0700200798002e0090000000e000cf
:1074280003003a000000eb00600f98008e00370060
:107438001e007800904078002e0090004158980077
:107448001e0fe8001e007800904078002e00900083
:10745800515898001e0fe8001e0078001040780070
:107468008080fb002e009000410098001e0fe8006d
:107478002e009000c00090001e0078001040780098
:107488000080fb004800dd00808040002e00900056
:10749800410098001e0fe8001e0078001040780098
:1074a8008080fb002e009000210098001e0fe8004d
:1074b800ae0090000000eb0090009800ae00900035
:1074c800314090000000a000b0409800ae0090004d
:1074d800214090000070a000a04098002e0190006c
:1074e8006000b8000009980011099800ae009000eb
:1074f8000040eb00805898002e0090009e009000fd
:10750800510898002e009000e008900000302000fc
:107518008080600000102000808f50001b003a001f
:107528002e009000200090000000e00003003a00c8
:10753800ae00900010002000a00098002e009000df
:1075480020009000f00f500003003600ae009000bd
:1075580000012000a00098002e009000200090005c
:107568000000e90080007800100020000100dd0024
:10757800800078002e00900021009800ae00900056
:10758800314090000000a100b04098002e0090000b
:10759800a00090002e009000310098001046800056
:1075a800900078002e0090000108780010468000b6
:1075b800ae009000010878001e4890000040e800e6
:1075c800104f98004e5090008080fb003e009000c5
:1075d8000100400030079800f14580003e0090000f
:1075e800008f4000be0090006e009000808f500019
:1075f800040031009e4890003e50900080cf50001b
:107608006eff39009e4890003e50900080cf500099
:10761800030032000000eb00600f980012003700f2
:10762800be0090006e009000808f5000d2fe39009e
:107638008e4890002e50900080cf500003003200fa
:107648008000eb00610f9800070037002e4890007b
:1076580012e8b7001e5090000080fb00c040880070
:1076680011002000610f98006e0890000080fa0059
:10767800000006000400fa00204798001046800029
:10768800000f78000e0037002e4090000004e00044
:10769800050032001e007800c05890002e4090006f
:1076a80080cf500004003a009e00780031409000de
:1076b8000010a100b04098001e007800100f78005c
:1076c8001e00e000f0ff3a000080fa00000006000b
:1076d8000400fa002047980031479800d0c5b3004d
:1076e800004f78001ac8bf00614060000004e00045
:1076f8000200320000c8b3001e4f70003040800006
:1077080050589000634060000004e00002003a0016
:10771800f0ceb3001e4f60003040800050589000fb
:1077280063406000e14f500002003a00e0cfb30030
:107738001e4f60001e80fb005025880014c8bf0043
:107748000080fb00b02488003e4090000080fb00d1
:107758004401dd002e4090008080fb00f0072000ef
:107768000080600000007100f024880094a4a80044
:107778000080fa00000006000600fa004047980062
:107788004e409000e94f500017003a0000a020003a
:10779800000f78001ac8bf00704060000004e000c5
:1077a8000200320040a02000000f78001ac8bf0075
:1077b8000080fb004400de006140600000c0ea0079
:1077c80061406000614060004401dd00a18120004b
:1077d80091407800f0ceb30000c060000240700015
:1077e8001ae8b7001600370080a02000000f7800c4
:1077f8001ac8bf000042b2000004e00002003200d4
:10780800c0a02000000f78001ac8bf000080fb004d
:107818004500de006140600000c0ea006140600091
:10782800614060004501dd00a181200091407800a1
:10783800f0cdb30000c06000024070001ae8b70045
:107848004e409000ed4f50001a003a003040800042
:10785800700090006101b8003040800090089000ee
:1078680000089000000151008181590030408000db
:107878004000900001002000800f5100818f5900c6
:107888000400360030408000c000900011079800c6
:1078980023003700304080007001900030408000a5
:1078a8009008900000089000000051001007980010
:1078b8001b0037003040800050019000e00190002c
:1078c80030408000900890000008900000015100ae
:1078d8008181590030408000400090000100200064
:1078e800800f5100818f590004003600304080001d
:1078f800c000900011079800090037003040800050
:10790800e0009000500090000001780030408000b6
:10791800900890000008900000005100100798009f
:107928004e409000ed4f500005003a003040800076
:10793800a00890001e007800110098000a00370087
:10794800304080003008900000017800304080000e
:107958009008900000089000000041008000780026
:107968001e007800110098009e0078000040eb008f
:10797800904098009e009000f03f20000081600039
:107988009e01780013007800f13f2000010161009a
:1079980001c02f000100600002007000800978001b
:1079a80030408000304090000080fb000000d10093
:1079b800614060009e017800930078000080fb0021
:1079c800610060004e01dd00f0ff2b008080600048
:1079d800828070008109780030408000304090003b
:1079e800614060009e017800930078000080fb00f1
:1079f800610060004b01dd00f07f2f008080600097
:107a080082807000810978009e007800110078005b
:107a180000f0a000800878000080fa00000006004e
:107a28000400fa0010468000000f78000b003700b1
:107a38001e007800a040900000c8b30000c060009d
:107a48000004e00003003a0010002000100798002e
:107a5800060037001e007800100f78001e00e000b6
:107a6800f3ff3a000000eb00100798001e0090009a
:107a78000080fa00000006003600f800809fbe0073
:107a8800829fbe00849fbe00869fbe003400f8001f
:107a980000c0b300a00188000a00fa007104800049
:107aa800f0fb2f00008060007004880082c4bf00d3
:107ab8000044b2000004e0001000320080c4bf009f
:107ac8000044b2000004e0000c0032000004200072
:107ad80000248800204080000000e9002040880041
:107ae800204080000000e00004003a0082c4a900a1
:107af800904280000000e800904288008cc4bf00db
:107b08000044b2000004e000100032008ac4bf0044
:107b18000044b2000004e0000c0032008cc4a9004c
:107b280000042000502488009142800000032000b7
:107b3800808f500005003a009142800000f020003c
:107b4800008060000010b000904288008cc4bf0024
:107b5800614060000004e000090032008ac4bf00f0
:107b6800614060000004e0000500320010002000c1
:107b7800502488008c04a9000000eb00a042880073
:107b88008cc4bf00684060000004e000720132004d
:107b98008ac4bf00684060000004e0006e01320043
:107ba800902480003007980080002000502488002e
:107bb80030408000405890000080fb00ef006000db
:107bc800f02480006f006000808f500061013a004f
:107bd8003e009000680060000000e00009003200ec
:107be80080a02000100798003e009000640060000c
:107bf8000000e0000b003200c0a020001007980031
:107c08000800370000a02000100798003e009000f0
:107c1800640060000000e0000200320040a0200084
:107c2800100798001e0090009000780000c0230004
:107c38008080600000802000808f500056003a004d
:107c48009e009000f03f200011006000200798007f
:107c58003440800030408000000990009009900076
:107c68002e009000010020000200400083804800a0
:107c7800000a9800110a9800314080000000eb00cb
:107c880080109800304080003040900062406000d2
:107c98000004e000050032003140800031409000cf
:107ca8000010a100b0409800040037003140800067
:107cb800314090000010a000b04098003040800093
:107cc80000589000f04f50000a0032003040800009
:107cd8008058900000c2b30080cf500005003200e9
:107ce800304080008058900000c3b30080cf50001f
:107cf80012003a003040800000099000900990007e
:107d0800304080007000900001002000800f51007a
:107d1800818f59000f013900324080006000b8009f
:107d2800000998001109980031408000015890001e
:107d38000040e80080589800060137003040800075
:107d4800c00090002e009000808f500009003e0077
:107d58003040800000099000900990003040800079
:107d6800e000900050009000800f5100818f590072
:107d7800f800390031408000214090000060a000e8
:107d8800a040980031408000015890000040e80071
:107d980080589800ef0037001e009000900078008f
:107da80000c023008080600000c02000808f500049
:107db800070032001e0090009000780000c02300e9
:107dc8008080600000c02200808f500036003a009a
:107dd8009e009000f03f20001100600020079800ee
:107de80034408000304080000009900090099000e5
:107df8002e0090000100200002004000838048000f
:107e0800000a9800110a9800314080000000eb0039
:107e18008010980030408000304090006240600040
:107e28000004e0000500320031408000314090003d
:107e38000010a100b04098000400370031408000d5
:107e4800314090000010a000b04098003040800001
:107e5800c00090002e009000808f500009003e0066
:107e68003040800000099000900990003040800068
:107e7800e000900050009000800f5100818f590061
:107e8800b400390031408000214090000060a0001b
:107e9800a040980031408000015890000040e80060
:107ea80080589800ab0037001e00900090007800c2
:107eb80000c023008080600000802200808f500076
:107ec80065003a0031408000314090000020a00059
:107ed800b040980031408000011090000000e80098
:107ee8008010980030408000505890006340600037
:107ef8000080fb00400798004e009000e10f500002
:107f08004c0032004e009000e10f500004003c008d
:107f18004e0090000000e000190032008d0037008c
:107f28004e009000e20f5000040032004e00900016
:107f3800e30f5000220032008600370030408000f6
:107f48008010900000712200808f50008100360060
:107f58003140800070c1b300e05898003240800082
:107f6800304080000058900080407800f0c0b30096
:107f780000c06000f040b300005998007500370059
:107f88003040800000109000f40f5000710036005f
:107f98003140800070c1b300e05898003240800042
:107fa800304080000058900080407800f0c0b30056
:107fb80000c06000f040b300005998006500370029
:107fc80030408000405890000004e0001000350068
:107fd8003040800000109000e30f50005d00360034
:107fe8003140800070c1b300e058980032408000f2
:107ff800304080000058900080407800f0c0b30006
:1080080000c06000f040b3000059980051003700ec
:1080180031408000214090000060a000a0409800fe
:1080280031408000015890000040e80080589800d6
:108038004800370031408000214090000060a000d7
:10804800a040980031408000015890000040e800ae
:10805800805898003f0037001e009000900078007c
:1080680000c023008080600000802300808f5000c3
:1080780010003a0031408000214090000030a000fc
:10808800a04098003140800010c1b300e05898002b
:1080980032408000304080000058900080407800d6
:1080a800f0c0b30000c06000f040b3000059980071
:1080b800280037003240800022409000674060006e
:1080c8000040e80067406000a2409000e74160007f
:1080d80080cfb30080c0600083c070002141980049
:1080e8003040800020409000674060000080fb0026
:1080f800e20f50001700340031408000214090000a
:108108000030a000a040980031408000214090003d
:108118000040a000a04098003140800030c1b3006a
:10812800e0589800324080003040800000589000ad
:1081380080407800f0c0b30000c06000f040b30099
:1081480000599800f00f20007024880020002000bb
:108158005024880041f607008cc4bf0064406000ca
:108168000004e000400032008ac4bf0064406000a0
:108178000004e0003c003200400020005024880049
:1081880010468000100f78001d0037001e00780090
:10819800e00890000030200080806000003020005f
:1081a800808f5000070032001e007800e008900021
:1081b800003020008080600000102000808f500078
:1081c80009003a001e007800300090000000e0002e
:1081d800050032001e007800300090008000e900a1
:1081e8001e007800310098001e007800b040900012
:1081f8000120a100314098001e007800100f78007f
:108208001e00e000e1ff3a00818020001140780064
:108218000000a1008048780081802000114078008b
:108228000010a1008048780081802000114078006b
:108238000020a1008048780081802000114078004b
:108248000030a10080487800828020006000b800db
:108258001001980021019800818020000040eb0067
:10826800e0409800fdf507008cc4bf006240600044
:108278000004e0005c0032008ac4bf006240600075
:108288000004e0005800320020002000502488003c
:108298003240800022409000674060000040e800c3
:1082a80067406000a2409000e741600080cfb300c3
:1082b80080c0600083c07000214198003040800079
:1082c80020409000674060000080fb00e20f5000f3
:1082d8004500340031408000214090000030a0006b
:1082e800a0409800e14820009140780000c8b30001
:1082f80000c060000004e00003003200314080004c
:1083080000c2b300e05898008ec4bf000042b2001b
:108318000004e000030032003140800010c2b300c6
:10832800e05898008ec4bf00704060000004e00070
:10833800030032003140800020c2b300e0589800aa
:108348008ec4bf00684060000004e00003003200f3
:108358003140800030c2b300e05898008ec4bf009e
:10836800644060000004e0000300320031408000f7
:1083780040c2b300e05898008ec4bf00624060005d
:108388000004e000030032003140800050c2b30016
:10839800e05898008ec4bf00614060000004e0000f
:1083a800030032003140800060c2b300e0589800fa
:1083b800f00f200070248800314080002140900098
:1083c8000040a000a040980032408000304080006b
:1083d8000058900080407800f0c0b30000c06000f2
:1083e800f040b300005998000080fa003400f9000a
:1083f8004f03be004f02be004f01be004f00be003b
:088408003600f90000400600f7
:020000040000fa
:108410000000fa00616a20009140780000ccb300af
:1084200000c06000a040b300a6e6b700116d2000b8
:108430009140780000ccb30000c060005040b30011
:10844000d1e6b70020302300103a88000000eb008e
:10845000203a88000000eb0000168800000c200085
:10846000c0168800920507000000eb000016880087
:108470000000eb0020168800c4c2a900c4e2a900d5
:10848000000c200050458800600807000000eb0049
:1084900030448800100020000080fa000000060030
:1084a0000800fa007cc8bf000004e00013003a0096
:1084b000804d2000000f7800c000200010079800b9
:1084c0000e007800cf0707000000e0000b0032002c
:1084d0004e4090007ce8b700006529006508070061
:1084e0007cc8bf0085080700606829006108070094
:1084f0001000200030079800020037000000eb0059
:10850000300798003e0090000080fa00000006004e
:108510000400fa000000eb00100798000c00370080
:108520001e019000a14680001e00900000804000c7
:1085300010407800804078008088200000004100d2
:10854000014878001e0090000000e8001007980025
:108550001e009000ef0f5000f1ff34000000eb0010
:10856000000f78000a0037001e017800b146800035
:108570001e007800008040001040780080407800a5
:108580008089200000004100014878001e0fe800ab
:10859000f00020009e0f1000f3ff340010c3b30062
:1085a0008de8b70000c3b3008fe8b70081882000d2
:1085b00010002000d4060700808920008000780089
:1085c00020002000d00607000080fa00000006000e
:1085d0000200fa00c18c2000914078007cc8bf00e6
:1085e00080cf500027003a00904680006100600074
:1085f0000000e000230032007246800083468000c5
:108600004000200001002000800f5100818f5900a0
:108610001c003a007ec8bf000004e00019003a00c8
:1086200081c8bf000004e0001600320081c8bf000e
:108630000043b00095e8b70082c8bf000043b00017
:1086400097e8b7008188200010002000ae060700e0
:10865000906829000708070081c8bf0027080700a5
:10866000206a29000308070082c8bf00230807000a
:1086700060682900ff07070010002000000f780045
:1086800007003700406a2900fa070700516c2900eb
:10869000200020009c0607000000eb00000f78007f
:1086a0001e0078000080fa00000006000600fa00b4
:1086b0007fc8bf000080fb00010020001007980069
:1086c0002107980080c8bf000080fb004800dd0043
:1086d0006101b9001e009000ae0090000200700021
:1086e0008380700010079800210798001e019000f9
:1086f000ae01900000902100010020000200400027
:108700008380480010079800210798001e00900001
:10871000ae00900092022000030020003ce9070018
:1087200010079800210798001e009000ae009000ee
:10873000a20020000300200045e90700004f780058
:108740001e009000ae009000a20020000300200058
:108750002fe9070010079800210798001e407800b5
:108760000043b0009be8b7001e009000ae009000f0
:10877000a20020000300200035e90700004f780028
:108780001e009000ae009000a20020000300200018
:108790001fe9070010079800210798001e40780085
:1087a0000043b00099e8b7001e009000ae009000b2
:1087b000a20020000300200025e90700004f7800f8
:1087c0001e009000ae009000a200200003002000d8
:1087d0000fe9070010079800210798001e40780055
:1087e0000043b00098e8b70080892000800078003e
:1087f00020002000440607000080fa000000060068
:108800000800fa007fc8bf000080fb0001002000c4
:10881000200798003107980080c8bf000080fb0047
:108820004800dd006101b9002e009000be009000fc
:1088300002007000838070002007980031079800c4
:10884000ae009000a07122000009b8002e00900038
:108850006000b9000302780000024200be009000f0
:10886000a07122000088b900000242008401780053
:1088700022079800330798002e009000be00900059
:108880004609dd004a00de0000007100ca08de0073
:1088900020079800310798000000eb00000f7800d7
:1088a000160037002e009000be009000a2002000ad
:1088b00003002000e6e80700204798002e00900003
:1088c000be009000a200200003002000d0e80700b6
:1088d0002007980031079800a00020001e015000da
:1088e0002e4090000043b000804078008089200036
:1088f00000004100014878001e0fe80042002000ff
:108900009e0f1100e7ff340080892000800078006e
:1089100020002000fc0507000080fa00000006008f
:108920000400fa00d116800000042000008f6000cf
:108930005145800000042000008060009e0f500020
:108940000f00320051458000f0fb2f0000806000d6
:1089500050458800504580001e007000504588003a
:10896000504580004600de00610060000004e00029
:1089700003003200100020001007980002003700aa
:108980000000eb00100798001e0090000080fa0025
:10899000000006000400fa00d11680000008200044
:1089a000008f6000514580000008200000806000ba
:1089b0009e0f50000f00320051458000f0f72f004d
:1089c0000080600050458800504580001e00700007
:1089d00050458800504580004700de00610060007f
:1089e0000004e0000300320010002000100798008f
:1089f000020037000000eb00100798001e009000f6
:108a00000080fa00000006000800fa00d043800051
:108a10000000e00002003a0080bb2000d043880044
:108a2000d04380000000e900d0438800304480003b
:108a3000e10f500003003e00c442a900c462a90037
:108a40006800370030448000e60f500003003e000d
:108a5000c442a800c462a80062003700304480000d
:108a6000f50f500022003e00d04380000000e000df
:108a70005c003a00c4c2bf000080fb004200de0080
:108a80000004a2006140600061406000614060003d
:108a9000614060004201dd00412c200091407800df
:108aa000b0cfb30000c0600002407000c4e2b70065
:108ab000c4c2bf000080fb004200de000004a20030
:108ac00061406000614060006140600061406000a2
:108ad0004301dd00412c20009140780070cfb300ad
:108ae00000c0600002407000c4e2b7003d003700e3
:108af000d04380000000e0001d003a00c4c2bf0067
:108b00000080fb004200de000004a2006140600023
:108b10006140600061406000614060004201dd0032
:108b2000412c200091407800b0cfb30000c060001d
:108b300002407000c4e2b700c4c2bf000080fb0066
:108b40004200de0061406000614060004301dd00e2
:108b5000412c20009140780070cfb30000c060002d
:108b600002407000c4e2b70020032000d043880018
:108b70001000200001002000008fbe00150037000b
:108b8000a0a62000010020002007980031079800cf
:108b90002e009000be00900061005000e080580060
:108ba00020079800310798002e019000be01900028
:108bb0000080eb008080eb00800f5100818f590016
:108bc000f3ff3a000080eb008080eb001e0f4000b6
:108bd0005e9748001e00be00e00f5000e08f580076
:108be000e7ff3a000080fa00000006000e00fa00dd
:108bf00085ff0700c18c2000914078007cc8bf0031
:108c000080cf500004003a00904680006100600070
:108c10000000e00009003a007cc8bf000004e0004a
:108c200006003200606d2900920607000000eb008c
:108c3000304488000040eb007ce8b70030448000fe
:108c40006101b80052079800630798006001200096
:108c5000010020005e019000ee019000800f5100a5
:108c6000818f59002d023e005e009000ee009000c2
:108c70000060010016003700190037001e003700a1
:108c80004500370054003700770037008600370072
:108c90008e003700b5003700c4003700e70037000a
:108ca000f6003700f9003700200137002f013700a8
:108cb000520137006101370064013700a601370017
:108cc000b5013700da013700e90137001502370036
:108cd0000ffe07001000200030448800110237000a
:108ce000effd07000000e0000e023200200020002f
:108cf000304488000b0237000040eb007ee8b700ec
:108d000020c0b3007fe8b700c18c200091407800fc
:108d10007cc8bf0080cf500002023a00904680001d
:108d2000610060000000e000fe013200904680001b
:108d3000620060000000e000fa013a007cc8bf0059
:108d40002200200003002000e1872000fc0507002e
:108d5000004f98000e4890000004e00003003a0025
:108d60003000200030448800ee013700e06f290019
:108d7000400607000e4890000080fb008d060700ab
:108d8000606829003b06070061712900200020006f
:108d9000dd040700e3013700c18c2000914078001a
:108da0007cc8bf0080cf5000de013a0090468000b2
:108db000610060000000e000da01320090468000af
:108dc000620060000000e000d6013a004000200090
:108dd00030448800d3013700c18c200091407800d6
:108de0007cc8bf0080cf5000ce013a009046800082
:108df000610060000000e000ca013200904680007f
:108e0000640060000000e000c6013a007cc8bf00ba
:108e10004200200003002000e18720009d0507009c
:108e2000004f98000e4890000004e00003003a0054
:108e30005000200030448800ba01370070722900c9
:108e40000c0607000e4890000080fb005906070042
:108e50006068290007060700e17329002000200050
:108e6000a9040700af013700c18c200091407800b1
:108e70007cc8bf0080cf5000aa013a009046800015
:108e8000610060000000e000a60132009046800012
:108e9000640060000000e000a2013a0060002000d1
:108ea000304488009f013700c9fd07000000e00042
:108eb0000300320070002000304488009901370020
:108ec00060012000304488009601370040c3b300a1
:108ed0007ee8b70020c0b3007fe8b700c18c200057
:108ee000914078007cc8bf0080cf50008d013a00cf
:108ef00090468000610060000000e00089013200bf
:108f000090468000620060000000e00085013a00a9
:108f10007cc8bf002200200003002000e187200061
:108f200087050700004f98000e4890000004e000fd
:108f300003003a00800020003044880079013700a7
:108f4000f0742900cb0507000e4890000080fb005c
:108f50001806070060682900c6050700617129002e
:108f600020002000680407006e013700c18c20003b
:108f7000914078007cc8bf0080cf500069013a0062
:108f800090468000610060000000e0006501320052
:108f900090468000620060000000e00061013a003d
:108fa00090002000304488005e013700c18c200012
:108fb000914078007cc8bf0080cf500059013a0032
:108fc00090468000610060000000e0005501320022
:108fd00090468000640060000000e00051013a000b
:108fe0007cc8bf003200200003002000e187200081
:108ff00028050700004f98000e4890000004e0008c
:1090000003003a00a00020003044880045013700ea
:1090100070762900970507000e4890000080fb003d
:10902000e40507006068290092050700e173290044
:1090300020002000340407003a013700c18c2000d2
:10904000914078007cc8bf0080cf500035013a00c5
:1090500090468000610060000000e00031013200b5
:1090600090468000640060000000e0002d013a009e
:10907000b0002000304488002a0137008bfd070033
:10908000c0002000304488002601370070c3b300c0
:109090007ee8b70020c0b3007fe8b700c18c200095
:1090a000914078007cc8bf0080cf50001d013a007d
:1090b00090468000610060000000e000190132006d
:1090c00090468000620060000000e00015013a0058
:1090d0007cc8bf002200200003002000e1872000a0
:1090e00017050700004f98000e4890000004e000ac
:1090f00003003a00d0002000304488000901370006
:10910000e07729005b0507000e4890000080fb0017
:10911000a80507006068290056050700617129004d
:1091200020002000f8030700fe003700c18c20005b
:10913000914078007cc8bf0080cf5000f9003a0011
:1091400090468000610060000000e000f500320001
:1091500090468000620060000000e000f1003a00ec
:10916000e000200030448800ee003700c18c200071
:10917000914078007cc8bf0080cf5000e9003a00e1
:1091800090468000610060000000e000e5003200d1
:1091900090468000640060000000e000e1003a00ba
:1091a0007cc8bf003200200003002000e1872000bf
:1091b000b8040700004f98000e4890000004e0003b
:1091c00003003a00f000200030448800d50037004a
:1091d00060792900270507000e4890000080fb00f9
:1091e000740507006068290022050700e173290063
:1091f00020002000c4030700ca003700c18c2000f3
:10920000914078007cc8bf0080cf5000c5003a0074
:1092100090468000610060000000e000c100320064
:1092200090468000640060000000e000bd003a004d
:109230000001200030448800ba00370070fd0700ac
:109240001001200030448800b600370020c3b3006e
:109250007ee8b70030c0b3007fe8b700b0fd07007c
:109260000000e0000900320030c0b3007fe8b70022
:10927000a8c8bf000080fb004300de006140600022
:109280000004a20080e8b7000f003700c1fd07000e
:109290000000e0000900320040c0b3007fe8b700e2
:1092a000a8c8bf000080fb004400de0061406000f1
:1092b0000004a20080e8b70003003700700020001f
:1092c0003044880097003700c18c2000914078001e
:1092d0007cc8bf0080cf500092003a0090468000ca
:1092e000610060000000e0008e00320090468000c7
:1092f000620060000000e0008a003a007cc8bf0005
:109300003200200003002000e18720008c040700c9
:10931000004f98000e4890000004e00003003a005f
:1093200020012000304488007e003700d07a2900d8
:10933000d00407000e4890000080fb001d050700c8
:1093400060682900cb04070061712900200020001b
:109350006d03070073003700c18c20009140780036
:109360007cc8bf0080cf50006e003a00904680005d
:10937000610060000000e0006a003200904680005a
:10938000620060000000e00066003a00300120004a
:109390003044880063003700c18c20009140780081
:1093a0007cc8bf0080cf50005e003a00904680002d
:1093b000610060000000e0005a003200904680002a
:1093c000640060000000e00056003a00a0cab3004c
:1093d0007ee8b7007cc8bf00120020000300200018
:1093e000e18720002b040700004f98000e489000f2
:1093f0000004e00003003a004001200030448800ef
:1094000048003700507c29009a0407000e4890005d
:109410000080fb00e704070060682900950407004e
:10942000e173290020002000370307003d003700ca
:10943000c18c2000914078007cc8bf0080cf5000d4
:1094400038003a0090468000610060000000e000b3
:109450003400320090468000640060000000e000ac
:1094600030003a0050012000304488002d003700c1
:10947000e18720009140780020c3b30080cf5000e6
:1094800023003a007fc8bf00e34f50000f003a00ae
:10949000a8c8bf000080fb004300de006140600000
:1094a0000004a20061406000614060004301dd00f3
:1094b000818a20009140780070cfb30000c0600026
:1094c00002407000a8e8b700110037007fc8bf0055
:1094d000e44f50000e003a00a8c8bf000080fb0017
:1094e0004400de00614060000004a20061406000b2
:1094f000614060004401dd00818a200091407800d5
:10950000f0ceb30000c0600002407000a8e8b700d1
:109510007000200030448800020037000000eb009b
:10952000304488001000200001002000008fbe00a1
:1095300015003700a0a62000010020002007980099
:10954000310798002e009000be009000610050008e
:10955000e080580020079800310798002e01900005
:10956000be0190000080eb008080eb00800f510076
:10957000818f5900f3ff3a000081eb008081eb00fe
:109580001e0f41005e9749001e00be00e00f500014
:10959000e08f5800e7ff3a000080fa000000060064
:1095a0000e00fa00004f780011079800220798007b
:1095b00034079800450798001e0090006007980047
:1095c000ee009000f18f50006f0032006e009000ae
:1095d000f10f50001a003e00ee009000e88f50009e
:1095e0005f0032006e009000e80f50000a003e005d
:1095f000ee009000e38f50007a0039006e0090007a
:10960000e40f500074003600ee009000e78f500029
:1096100071003200730037006e009000ee0f5000b2
:109620004c003200ee009000f08f500051003200ec
:109630006e009000ed0f50004300320069003700cb
:1096400040062000ee009000808f50001b0032008a
:1096500040062000ee009000808f50000a003e007f
:109660006e009000f30f500051003200ee009000a9
:10967000f38f5000490039006e009000f40f500045
:10968000500032005700370070062000ee009000b6
:10969000808f500005003e0060062000ee00900024
:1096a000808f5000250031001b0037006e009000b5
:1096b000e10f4000480032004a0037003e019000b0
:1096c000ce0190006000200001002000800f5100ba
:1096d000818f590043003a002e00900040409000d6
:1096e0007ce8b7002000200030448800c07d2900bd
:1096f000e00307007cc8bf00000407006068290081
:10970000dc03070060682900da030700110020006d
:1097100051079800350037000040eb007ce8b700a7
:109720000000eb003044880010812900d1030700bd
:1097300010002000500798002c0037001100200076
:1097400051079800290037001000200050079800aa
:109750002600370011002000510798002300370031
:1097600080832900c30307001000200050079800e1
:109770001e003700b0862900be030700110020003c
:109780005107980019003700f0892900b903070034
:10979000100020005007980014003700308d290079
:1097a000b403070011002000510798000f00370094
:1097b00020912900af0307001000200050079800f7
:1097c0000a00370010942900aa03070011002000a6
:1097d000510798000500370010002000500798003e
:1097e000020037008000eb00510798005e009000f7
:1097f0000080fa00000006000000fa0004fb0700e9
:10980000e10f5000030032009096290099030700f1
:10981000ffff37006000b800c9e70700e10f500004
:1098200003003a00e09a2900920307000300370082
:10983000209e29008f030700ffff3700bee80700c6
:08984000eafc0700fdff370000
:020000040000fa
:109848000400fa00004f780011479800e002a900d0
:10985800e022a900e042a900e062a900e082a90094
:10986800e0a2a900e0c2a900e0e2a900c9e2a900bb
:10987800d8a2a900dca2a9009e40780061c06000bf
:10988800c700dd00cdc2bf000074a1000140700018
:10989800cde2b7001e40900061406000614060006a
:1098a8006140600061416000412e200091407800d5
:1098b800e0cfb30000c0600002407000e4e2b700ef
:1098c8001e4090000080fb000000d1006140600055
:1098d80061406000614060006140600000414000fc
:1098e800412e200091407800d0cfb30000c0600026
:1098f80002407000e4e2b7001e4090000080fb00c8
:109908004200de006140600061406000614060002c
:10991800614060004201dd00412e20009140780046
:10992800b0cfb30000c0600002407000e4e2b700ae
:109938001e4090000080fb004300de006140600094
:109948006140600061406000614060004301dd00eb
:10995800412e20009140780070cfb30000c0600015
:1099680002407000e4e2b7001e4090000080fb0057
:109978004400de00614060006140600061406000ba
:10998800614060004401dd00412e200091407800d4
:10999800f0ceb30000c0600002407000e4e2b700ff
:1099a8001e4090000080fb004500de006140600022
:1099b8006140600061406000614060004501dd0079
:1099c800412e200091407800f0cdb30000c0600027
:1099d80002407000e4e2b7001e4090000080fb00e7
:1099e8004600de0061406000614060006140600048
:1099f800614060004601dd00412e20009140780062
:109a0800f0cbb30000c0600002407000e4e2b70091
:109a18001e4090008040eb00214798000004e000c1
:109a280002003d0010c0b300204798002e4090006f
:109a3800c700dd00e4c2bf000074a100014070004f
:109a4800e4e2b7000000000000000000dc82a8008b
:109a580000000000000000000000000000000000fe
:109a680000000000000000000000000000000000ee
:109a780000000000dc82a900e002a800e022a800a3
:109a8800e042a800e062a800e082a800e0a2a800e6
:109a9800e0c2a800e0e2a800c9e2a800d8a2a80095
:109aa8000080fa00000006002600fa0002022000ea
:109ab800010220008085200020e407000040eb0020
:109ac80078e8b700dc82a900dca2a900e002a900be
:109ad800e022a900e042a900e062a900e082a90012
:109ae800e0a2a900e0c2a900e0e2a900d8a2a9006a
:109af800c9e2a900d882a900800220000100200044
:109b0800600f9800710f980017003700a0a620007a
:109b18000100200000179800111798000e109000ff
:109b28009e10900061005000e080580000179800d7
:109b3800111798000e1190009e1190000080eb0004
:109b48008080eb00800f5100818f5900f3ff3a00ad
:109b58006e089000fe08900061005000e0805800f8
:109b6800600f9800710f98006e089000fe08900032
:109b7800e00f5000e08f5800e4ff3a00cde2a90062
:109b8800e402a800e422a800e442a900e462a900d3
:109b9800e482a900e4a2a900e4c2a900e4e2a900c1
:109ba80000000000000000000040eb004067980043
:109bb80027003700dc82a800a00120000100200057
:109bc800400f9800510f98004e089000de08900052
:109bd80061005000e0805800400f9800510f980035
:109be8004e099000de0990000080eb008080eb00b9
:109bf800800f5100818f5900f3ff3a00dc82a900e1
:109c08002008200001002000200f9800310f980044
:109c18002e089000be08900061005000e0805800b7
:109c2800200f9800310f98002e099000be0990006f
:109c38000080eb008080eb00800f5100818f59007d
:109c4800f3ff3a004e6090000040e800406798003b
:109c58004e609000e24f5000d6ff360081c3b3003b
:109c68000040eb00f6fe070020082000010020005d
:109c7800000f9800110f98000e0890009e089000a1
:109c880061005000e0805800000f9800110f980004
:109c98000e0990009e0990000080eb008080eb0088
:109ca800800f5100818f5900f3ff3a0061c0b30063
:109cb8000040eb00e2fe0700200820000100200021
:109cc80060079800710798006e009000fe009000f1
:109cd80061005000e0805800600798007107980004
:109ce8006e019000fe0190000080eb008080eb0088
:109cf800800f5100818f5900f3ff3a00c1c0b300b3
:109d08000040eb00cefe07002008200001002000e4
:109d180040079800510798004e009000de00900020
:109d280061005000e08058004007980051079800f3
:109d38004e019000de0190000080eb008080eb0077
:109d4800800f5100818f5900f3ff3a0011c0b30012
:109d58000040eb00bafe07002000200001002000b0
:109d6800008fbe0015003700a0a6200001002000cb
:109d780020079800310798002e009000be00900040
:109d880061005000e08058002007980031079800d3
:109d98002e019000be0190000080eb008080eb0057
:109da800800f5100818f5900f3ff3a000080eb00cb
:109db8008080eb001e0f40005e9748001e00be002a
:109dc800e00f5000e08f5800e7ff3a000080fa00eb
:109dd800000006001600fa0021c0b3000040eb00a6
:109de80097fe07002000200001002000600798006f
:109df8007107980017003700a0a620000100200076
:109e0800000f9800110f98000e0890009e0890000f
:109e180061005000e0805800000f9800110f980072
:109e28000e0990009e0990000080eb008080eb00f6
:109e3800800f5100818f5900f3ff3a006e009000a7
:109e4800fe00900061005000e08058006007980014
:109e5800710798006e009000fe009000e00f50001f
:109e6800e08f5800e4ff3a000040eb00505798009c
:109e7800310037005e5090008080fb008085200014
:109e880000804000104078000004e0000f003a0015
:109e98005e50900040579800090037004e509000df
:109ea8008080fb00808520008080400000c2b300d5
:109eb800804878004e5090000040e80040579800d5
:109ec8004e509000ef4f5000f4ff36005e50900067
:109ed8008080fb0080852000008040009040780052
:109ee80010c0b30056fe0700200820000100200023
:109ef80040079800510798004e009000de0090003f
:109f080061005000e0805800400798005107980011
:109f18004e019000de0190000080eb008080eb0095
:109f2800800f5100818f5900f3ff3a005e50900076
:109f38000040e800505798005e509000ef4f5000e6
:109f4800ccff360001ccb3000040eb003cfe07001c
:109f58002008200001002000200798003107980001
:109f68002e009000be00900061005000e080580074
:109f780020079800310798002e019000be0190003c
:109f88000080eb008080eb00800f5100818f59002a
:109f9800f3ff3a0000c1b300505798002c00370077
:109fa8005e5090008080fb0080852000008040008b
:109fb800104078000004e0000f003a00de509000e6
:109fc80041579800090037004e5090008080fb00f0
:109fd800808520008080400000c2b300804878005f
:109fe8004e5090000040e800405798004e509000b6
:109ff800ff4f5000f4ff36005e5090008080fb0059
:10a0080080852000008040009040780010c0b30098
:10a018000bfe07002008200001002000008fbe0072
:10a028000080eb008080eb001e0f40005e97480028
:10a038000080eb008080eb00be0f1000ae8f180090
:10a04800f7ff3a005e5090000040e8005057980033
:10a058005e509000ff4f5000d1ff36000080fa009c
:10a06800000006000800fa0011c0b3000040eb0031
:10a07800f3fd07002000200001002000008fbe0033
:10a0880015003700a0a62000010020002007980036
:10a09800310798002e009000be009000610050002b
:10a0a800e080580020079800310798002e019000a2
:10a0b800be0190000080eb008080eb00800f510013
:10a0c800818f5900f3ff3a000080eb008080eb009d
:10a0d8001e0f40005e9748001e00be00e00f5000b3
:10a0e800e08f5800e7ff3a0002022000010220003a
:10a0f8008085200091e207000080fa000000060039
:10a108000600fa0010079800210798000040eb00ad
:10a11800004f78000040eb00104798001e009000a8
:10a12800e20f50000b003a00010037001e4fe80014
:10a138009e80fb0080852000008040001040780051
:10a148000004e00003003200f0c0b3009e4f10008e
:10a15800f6ff36001e81fb001e4090000080fb00c9
:10a16800800078002e0090000080400010407800a9
:10a178008040780080852000000041000148780078
:10a188001e4fe8001e4090000040e800104798006d
:10a198001e80fb008000e9008085200000804000d0
:10a1a800104078000004e00003003200e0c1b30072
:10a1b8009e4f1000e7ff360006ff07000080fa00f8
:04a1c800000006008d
:020000040000fa
:10a1cc000800fa00204798002207980033079800ef
:10a1dc006000b80070468800814688000040eb00a3
:10a1ec00d2e8b7002e409000cce8b70000468000c3
:10a1fc00000f78001e007800680f40001e007800e9
:10a20c00104078000080fb00404688001e0fe800dc
:10a21c00414680001e007800104078000080fb0052
:10a22c004800dd0000807000404688001e0fe800ea
:10a23c001e007800104078000080fb00504688001b
:10a24c001e0fe800514680001e0078001040780078
:10a25c000080fb004800dd00008070005046880044
:10a26c001e0fe800d208a8006400200005002000a2
:10a27c00828c2000410620002e409000c5fc070077
:10a28c00100020000080fa00000006001200fa0006
:10a29c0040479800310798004207980054079800ef
:10a2ac0065079800c18c2000914078004e409000ca
:10a2bc0080cf5000030032000000eb0070079800c4
:10a2cc004a0037003e009000000f98000e089000e6
:10a2dc00e10f5000110032000e089000e70f500003
:10a2ec00010032003f003700ccc8bf001400200032
:10a2fc0005002000c28c200051062000a5fc0700a0
:10a30c000040eb00d2e8b7000040eb00cce8b7000f
:10a31c001000200070079800340037004e009000a9
:10a32c000000e0002c0032005e019000ee01900075
:10a33c00a000200001002000800f5100818f5900e7
:10a34c0025003a004e0090001000be00008fbe00a9
:10a35c004e009000e040900010c8b30080cf500039
:10a36c000b003a00d248a9001e00be0070468800bf
:10a37c0081468800ccc8bf004400200005002000a6
:10a38c000e0178007106200082fc07000f003700d8
:10a39c004e00900060409000e14f500008003a00e1
:10a3ac00d228a900ccc8bf00440020000500200022
:10a3bc000e0178006106200076fc070003003700d0
:10a3cc000000eb0070079800080037001000200018
:10a3dc0070079800050037000000eb00700798002c
:10a3ec00020037000000eb00700798007e00900020
:10a3fc000080fa00000006000400fa00000f78004c
:10a40c0090468000610060000000e00003003a000c
:10a41c000000eb001007980018003700ccc8bf00f4
:10a42c000004e000130032001e00e00011003200b6
:10a43c001e0078009000780040468000808f50000d
:10a44c000c003a001e0078009000900050468000ee
:10a45c00808f500007003a00c18c2000914078009a
:10a46c001e00780041409800100020001007980052
:10a47c00020037000000eb00100798001e0090004f
:10a48c000080fa00000006000c00fa00204798003b
:10a49c00210798003207980043079800c18c2000d0
:10a4ac00914078002e40900080cf500004003a007c
:10a4bc0090468000610060000000e00003003a005c
:10a4cc0010002000500798001700370090468000bd
:10a4dc00640060000000e000030032002000200057
:10a4ec005007980010003700d248a8006000b80050
:10a4fc0070468800814688002e0190003e02900034
:10a50c00ce02900011c8b3002e409000b2e40700b8
:10a51c00004f78001e04e00001003200d248a90070
:10a52c001e80fb00500798005e0090000080fa002f
:10a53c00000006000c00fa00204798002107980044
:10a54c003207980043079800c18c20009140780096
:10a55c002e40900080cf500004003a0090468000be
:10a56c00610060000000e00003003a0010002000d1
:10a57c00500798001400370090468000620060007d
:10a58c000000e0000300320020002000500798007b
:10a59c000d003700d228a8002e0190003e0290003a
:10a5ac00ce02900011c0b3002e409000e0eb0700eb
:10a5bc00004f78001e04e00001003200d228a900f0
:10a5cc001e80fb00500798005e0090000080fa008f
:04a5dc000000060075
:020000040000fa
:10a5e0000200fa0087c0bf000044b2000004e0008f
:10a5f000fcff3200b0118000004f780087c0a90036
:10a600001e00fb000080fa00000006000000fa00b7
:10a6100040042000c01188000000eb008011880079
:10a620003062a8000000eb009011880031e2a80021
:10a630003342a80087c0a9000080fa00000006008d
:10a640000200fa0087c0bf000044b2000004e0002e
:10a650000300320010002000000f780002003700d5
:10a660000000eb00000f78001e0078000080fa0068
:10a67000000006000600fa001007980002003700ec
:10a680001e407800120007001e0090001040780065
:10a69000004f78001e407800404798004e409000e0
:10a6a0000004e0000200320010c0b30040479800f0
:10a6b0004e4090009e0090008100e8001107980035
:10a6c0000004e000eeff3a000080fa0000000600ff
:10a6d0000200fa00004f78001e00fb00a011880065
:10a6e0000000000033c2bf00614060000004e000d1
:10a6f000fcff32000080fa00000006000400fa00af
:10a70000204798002e409000004f780030c6b300dc
:10a710009e4f1000060036001e80fb0042062000ff
:10a72000110009000280d8000043b000e8ff0700d4
:10a730009e4178001e80fb004206200011000900a7
:10a740000280d8008080fb00400620000088b9000d
:10a7500000c05100004f780090c0b3009e4f100021
:10a76000060036001e80fb00a20020001100090038
:10a770000280d8000043b000d5ff07009e4178005a
:10a780001e80fb00a2002000110009000280d800fa
:10a790000080fb006a00b90000c05100004f780043
:10a7a0001e4078000043b000c9ff07000080fa0097
:10a7b000000006000400fa00100798001e00900038
:10a7c000000f78001e0090004480de006f006000e3
:10a7d000100798009e00900040a229006140780078
:10a7e000bbff07009e0078006f8060001007980094
:10a7f0009e00900040a2290061407800b4ff07004d
:08a800000080fa0000000600d0
:020000040000fa
:10a80800d408000004000000020000002e963f005b
:10a81800960000007a0800003200000000000000e6
:10a82800ac0800001000000002000000e6504c00d8
:10a83800510000000000d800040c000000000000d7
:10a8480000000000bc0800000c000000020000002e
:10a8580000000000000000000000000000000000f0
:10a86800000a0000100000000000000000080000be
:10a878005800000000000000c80800000c0000009c
:10a88800000000005808000022000000000000003e
:10a89800da080000060000000200000000020000c4
:10a8a80000000000d80800000200000000000000be
:04a8b800000000009c
:020000040000fa
:04a8bc000000fe009a
:00000001FF
